:020000041000EA
:10000000002008205D0100101B0100101D010010E0
:100010001101001011010010110100101101001058
:100020001901001019010010190100101F01001022
:10003000110100101901001021010010230100100E
:100040001101001011010010110100101101001028
:100050001101001011010010110100101101001018
:100060001101001011010010110100101101001008
:1000700011010010110100101101001011010010F8
:1000800011010010110100101101001011010010E8
:1000900011010010110100101101001011010010D8
:1000A00011010010110100101101001011010010C8
:1000B00011010010110100101101001011010010B8
:1000C00011010010110100101101001011010010A8
:1000D0001101001011010010110100101101001098
:1000E0001101001011010010110100101101001088
:1000F0001101001011010010110100101101001078
:100100001101001011010010110100101101001067
:10011000EFF30580103800BE00BE00BE00BE00BE7A
:1001200000BE00BEF2EB887120A3001040A30010B7
:10013000A001001090A31AE7D3DEFFFF42012110B7
:10014000FF01000000B00000793512AB4FF0000055
:100150001E49086006C881F3088810474FF05040D8
:10016000006810B14FF00000F2E70DA40ECC00299A
:1001700002D000F012F8F9E71549164A002000E015
:1001800001C19142FCD11449884714498847144958
:10019000884700BEFDE701C901C29A42FBD3704700
:1001A00040A3001010010020080F002038B10010FB
:1001B000000008200000082038B1001000100820BE
:1001C00000100820000000007047000008ED00E06B
:1001D000080F0020E81E0020052F0010DD0200108F
:1001E000C52E0010F8B500BF0348044B834202D06F
:1001F000034B03B118477047080F0020080F002079
:1002000000000000064B0749C91A891048BF013198
:10021000491003D0044B0BB101481847704700BF89
:10022000080F0020080F00200000000010B5064C49
:10023000237843B9FFF7D8FF044B13B10448AFF359
:1002400000800123237010BD9010002000000000EA
:100250008474001008B5044B1BB104490448AFF383
:100260000080BDE80840CDE70000000094100020A9
:100270008474001010B582B00190074B074A0849FA
:1002800006F086F801AC204606F0F2FE002120467A
:1002900006F0F5FE02B010BD9D030010190300101A
:1002A000B0A2001038B504460D4606F018F82046F6
:1002B00006F05FF80849204606F074FB2B4614222E
:1002C0003A21204606F02EFB204606F04EF828463E
:1002D00002F02CFF38BD00BFD483001010B5A6B0CB
:1002E00001A8FFF7C7FF02F01DFF002408E008493E
:1002F00001A8FFF7D7FF4FF47A7000F0E3FF013455
:1003000014F0010FF3D0034901A8FFF7CBFFF2E788
:10031000887400108C74001038B5044618291ED05B
:1003200008D919292AD0202910D14A2106F0B5FE72
:10033000012008E014290BD0172905D119461648C9
:1003400007F076F8012038BD0020FCE70020FAE72E
:1003500003685A78492106F0A0FE0120F3E70368FC
:100360001A78492106F099FE63691D462268002328
:1003700092782C212046A8470120E4E70268002358
:10038000D2782C214569A84723685A78492120460C
:1003900006F083FE0120D6E70080084008B52C292E
:1003A0004DD011D82A294FD007D8282919D029296A
:1003B0005FD1104600F086FF3FE02B2959D110464F
:1003C000002100F06DFF38E04A2944D04B2949D084
:1003D00049294ED1003A18BF01220D2342EC40308A
:1003E0002BE02649264805F019FF05210D2000F0D5
:1003F00049F801210A2000F045F801210B2000F006
:1004000041F80E2000F05AF80C2000F057F80D20AB
:1004100000F054F80E204FF0010343EC44000C228E
:1004200043EC44200D2143EC441043EC400043ECEA
:1004300040104FF0000343EC4020012008BD10465F
:10044000002100F02DFFF8E702EB820250000021AE
:1004500000F026FFF1E7003A18BF01220C2342EC1E
:100460004030EAE7003A18BF01220E2342EC403048
:10047000E3E7012380F82730DFE700BF00127A00AE
:10048000008008400C4B03EB800253F8203083F0CF
:10049000400303F0C00302F5805CCCF80030C000DC
:1004A00000F1804000F52030416002F540524FF4E9
:1004B00080731360704700BF0480034008B54FF09D
:1004C000000242EC440042EC40000521FFF7DAFF55
:1004D00008BD00000FB400B583B0084802F026FE46
:1004E000049B3BB105A90191184602F02FFE044878
:1004F00002F01CFE012002F0E3FC00BF907400102B
:10050000A0740010EFF3108072B6064BD3E8CF1F33
:1005100001220029FAD1C3E8412F0029F6D1BFF307
:100520005F8F7047F31300200023034AC2E88F3F18
:1005300080F31088704700BFF313002070B50546A4
:100540000C461646FFF7DEFFE208A95C04F0070C34
:10055000012303FA0CF3194205D1DBB20B43AB5470
:10056000FFF7E2FF70BD21463046FFF7B3FFF8B555
:1005700005460F4614461E46FFF7C4FF00E001344F
:10058000B4420ED84FEAD40C15F80C1004F007034F
:1005900001229A401142F2D1D2B20A4305F80C204E
:1005A00001E04FF0FF34FFF7BFFF002C01DB2046D6
:1005B000F8BD002FFBD00698FFF78CFF054A107896
:1005C000431CDBB21370172B02D9134610221A708A
:1005D000704700BF600E002000B583B00146044B99
:1005E00000931F2318220348FFF7C1FF03B000BD8B
:1005F000A4740010241A00204FF0E022936843F006
:100600000053936070470000002305E0044A1A4439
:100610000021C2E88F1F01331F2BF7D9704700BF9D
:10062000E8130020064B9B68103043F82010BFF3FE
:100630005F8F00230349C1E88F3F82F31088704722
:1006400000ED00E0F11300200048704700E400E0F6
:1006500008B5FFF7F9FF002304E04FF0803240F8BF
:10066000042B01330C2BF8D962B608BD08B50388FA
:10067000DA0A1C2A06D15B050BD45B15023300EBAA
:10068000430008BD064B074A4FF48E71064802F03E
:100690001DFC03F5FF1303F5FF531F33EDE700BF08
:1006A000C0740010607E0010D874001008B5091ADC
:1006B00001F2FC7240F6FE739A4208D8081F11F04E
:1006C000010F04D1C0F34A0040F4604008BD034B61
:1006D000034A4FF48771034802F0F8FB4475001099
:1006E000547E0010D87400104209064B53F82220A3
:1006F00000F01F00012383401A4214BF0120002094
:10070000704700BF00E100E03AB1064B00F1600223
:1007100043F8221043F8201070472030014B43F873
:100720002010704700E100E008B50A4600F01F0302
:10073000012199404009FFF7E7FF08BD00F01F02C3
:100740004009012393404030014A42F8203070476D
:1007500000E100E0024B9B68103053F82000704726
:1007600000ED00E008B5FFF7F5FF034BC01A2F2896
:100770008CBF0020012008BD640E002070B5054626
:100780000C46EFF3108372B61E460F4BD3E8CF1F13
:1007900001220029FAD1C3E8412F0029F6D1BFF385
:1007A0005F8FFFF7D7FF094B984201D0A04205D1D8
:1007B000324621462846FFF735FF70BD044B054AF7
:1007C000ED21054802F082FBF11300201101001019
:1007D00074750010887E0010D87400102DE9F04F59
:1007E00087B000911546EFF3108372B69B467C4BA1
:1007F000D3E8CF1F01220029FAD1C3E8412F0029F5
:10080000F6D1BFF35F8F774B93F90040002C44DBA8
:10081000804604EB4407744B03EB870797F90610F7
:10082000704A1170714A926800F1100152F82190DB
:10083000A9EB03022F2A3ED96D4B994534D14FF4D1
:100840002143ADF80C304FEA440904EB4400664EF6
:1008500006EB800067490230FFF728FFADF80E0075
:100860004BF60153ADF81030FF238DF812308DF8A0
:100870001350009B0593A14406EB890306AA12E9D5
:10088000070083E8070047F001095A4649464046F9
:10089000FFF7C8FE07B0BDE8F08F574B574A4FF43B
:1008A000BE71574802F012FB564B544A40F2831176
:1008B000534802F00BFB29F001029246D31A524A28
:1008C000A2FB0312D20802EB4202B3EB820F0FD15C
:1008D00053460026DA79AA4212D993F90620002A53
:1008E0000DDB02EB42021E463F4B03EB8203F1E7B6
:1008F000464B424A4FF4CA71414802F0E7FA1E469D
:10090000A6B344F60103ADF80C304FF48F43ADF8B5
:100910000E3096F906309A46002B1ADA4BF6015043
:10092000ADF810008DF812A08DF81350009B0593C0
:100930003946301DFFF7BAFEB080B47104EB4404B1
:10094000294B03EB840306AA12E9070083E807009A
:100950009BE7301DFFF78AFE014604EB4402224B61
:1009600003EB8203181DFFF7A1FED9E74FF42143E3
:10097000ADF80C306300019304EB4406DFF8689097
:1009800009EB86061B49B01CFFF790FEADF80E0080
:100990005146301DFFF78AFEADF810004AF6AA2333
:1009A00052464946521A524153431B0D8DF812309C
:1009B0008DF8135000990591019B234409EB83099D
:1009C00006AB13E9070089E8070044F60103AAF81B
:1009D00000304FF48F43AAF8023047F0010954E782
:1009E000F1130020E01E0020640E002000ED00E066
:1009F00011010010940E0020AC750010707E0010E4
:100A0000D8740010D4750010ABAAAAAAFC75001007
:100A100038B540F00104344BE31A2F2B35D8EFF3EF
:100A20000581C9B2002937D0EFF3108E72B62F4B73
:100A3000D3E8CFCF0122BCF1000FF9D1C3E84C2F8E
:100A4000BCF1000FF4D1BFF35F8F4AF6AA23024630
:100A5000DFF894C06546521B524153431B0D4FFAB9
:100A600083FC234B9B6853F82130A3421BD0002307
:100A7000032B32D803EB43011B4A02EB810292F9AC
:100A80000620624520D00133F2E71A4B1A4A40F2A1
:100A90007F211A4802F01AFA194B174A40F28221B4
:100AA000164802F013FA124B9B68164A43F82120AD
:100AB000154B1A78827183F800C000230B4AC2E8F4
:100AC0008F3F8EF3108838BD074A02EB8101FF2467
:100AD0008C714BF601538B80EAE70C4B064A40F2CF
:100AE0009321064802F0F2F9640E0020F113002071
:100AF00000ED00E080760010387E0010D874001001
:100B0000A876001011010010E01E0020B47600103D
:100B100000B583B00146064B00930523002205482B
:100B2000FFF725FD002801DBC0F1330003B000BD55
:100B3000BC760010E41E0020014B0B44036070479C
:100B4000E813002010B50446FFF738FD01462046A3
:100B5000FFF7F2FFFF232371BFF35F8F10BD10B5C6
:100B60000446FFF72BFD01462046FFF7E5FFFF2374
:100B7000237100236371BFF35F8F10BD10B50D4C5F
:100B800009E00D4B0D4A1A210D4802F09FF920464D
:100B9000FFF7D8FF08340B4B9C4209D22368002B87
:100BA000F5D0012BEDD12046FFF7D9FF0834F2E74D
:100BB00010BD00BF000F0020D8760010C87E0010C6
:100BC000F8760010080F0020024B0B440360BFF3BF
:100BD0005F8F7047E813002010B504460120FFF72F
:100BE000FBFC01462046FFF7EFFF10BD0246EFF386
:100BF0000583DBB2103B990804D0034803F00303DC
:100C0000136070470148F9E700800B4000000B407B
:100C100000B5D0F828C0A2EB0C0E0B1D50F8233005
:100C2000A3EB0C039E4506D3D0F820C001238B40D4
:100C30001CEA030F02D1043140F8212000BD41EA33
:100C4000004070470D4B1A68EFF3108172B6D2E87E
:100C5000CFCF0120BCF1000FF9D1C2E84C0FBCF19D
:100C6000000FF4D1BFF35F8F1A680023C2E88F3FF3
:100C700081F3108840BF002000217047C01E002073
:100C80002DE9F04F85B003A8FFF7B0FF954B9842D0
:100C900014BF00230123039901EB8303924A52F806
:100CA00023402378994206D1054601228A4000F567
:100CB00041535A602CE18D4B8D4A92218D4802F0B0
:100CC00005F9D4F8149006EB46074FEAC70A09EB7A
:100CD000C707D7F808B0D7F80C80284600F0B6FB55
:100CE000B0EB0B0061EB0803002BC0F21A81B8F1E6
:100CF000000F64DB3B691A4600937F4B9A4230D069
:100D0000798889B2B4F90800FFF799FF7969009BE7
:100D10009847009001910099019A51EA02034ED040
:100D20001346002A29DABBEB010268EB0308BA601C
:100D3000C7F80C8039F90A70002FC0F2F280D4F89D
:100D400014E007EB47030EEBC3039968DB68511A05
:100D500068EB0303002BC0F2E480A4462CF8087F64
:100D600017E07A69136900921046984738B3009AE1
:100D70001368009353680193CDE7284600F066FBA3
:100D8000009B1A18019B43EB0108D0E79C463EF9F3
:100D90000B70002F0EDBBCF9003003EB43034FEA6E
:100DA000C30B0EEBC3039868D968101A68EB0101F6
:100DB0000029EBDA29F80A70ACF80060B1E039F9E3
:100DC0000A3023812369EFF3108272B6D3E8CF0F84
:100DD00001210028FAD1C3E8401F0028F6D1BFF353
:100DE0005F8FB4F9023029F80A3066802169002348
:100DF000C1E88F3F82F3108893E02369EFF31082FC
:100E000072B6D3E8CF0F01210028FAD1C3E8401F02
:100E10000028F6D1BFF35F8FB4F804800FFA88F88A
:100E20004FF6FF73A38021690023C1E88F3F82F34F
:100E300010881AE01F4630F90A60002E0FDBB7F960
:100E4000003003EB43034FEAC30A00EBC303996886
:100E5000DA68BCEB01016EEB0202002AEADAA7F8BD
:100E6000008030F9098020F80960B8F1000F5DDBDF
:100E7000606908EB48034FEAC30900EBC303D3F8EA
:100E800008C0D3F80CE004F10807B4F90860D4E70F
:100E90000023A37104F1080CB4F9083010E04FF0FE
:100EA000FF384FF0FF39C0E90289B4F908009842D1
:100EB00005D0ACF80020B4F90800C85323811346CC
:100EC000B3F1FF3F35D0616903EB4302D70001EB7B
:100ED000C20031F93220468816F4004FDFD1844633
:100EE000EDE700BF00800B40981E0020B477001093
:100EF000F47E0010E0770010810C0010284600F00E
:100F0000A5FA3F1A66EB0106012F76F1000628DAF2
:100F1000039A01239340EB63B4F90860002EBFF6F7
:100F2000D0AEA38813F4004F3FF467AFA379002B32
:100F3000AED1B4F90830002B13DB626903EB430335
:100F400002EBC3039F68DE68B6F1FF3F08BFB7F14D
:100F5000FF3FD3D03A46334603992846FFF758FE61
:100F6000CCE740BF05B0BDE8F08F00BFF8B5044640
:100F70000D4611460A4B984210D000262E440127F8
:100F800007FA05F525623046FFF7F8FB394630468B
:100F9000FFF7CAFB04F501542560F8BD0426EDE710
:100FA00000800B40F8B504460E4617461D46C1604A
:100FB000FFF704FB164B034423612770ABB2638138
:100FC0004FF05042127862704FF6FF722281A28079
:100FD000013B63804FF0000C08E00CF1FF300CEB9C
:100FE0004C0E636923F83E000CF1010CAC45F4D3C0
:100FF000084B9E4214BF0023012307EB8303064ADC
:1010000042F82340054A39463046FFF7AFFFF8BDA6
:10101000E813002000800B40981E0020810C001077
:1010200008B5054B1B690BB1034808BD034B044AC7
:101030006521044801F04AFFAC0E002044780010FE
:10104000DC7E0010E0770010F8B504469E4600698B
:10105000EFF3108172B6D0E8CF6F0125002EFAD1E0
:10106000C0E8465F002EF6D1BFF35F8FB4F902509F
:10107000666905EB4500C70006EBC000002D03DBE9
:1010800036F907C0A4F802C04FF0000C2369C3E88A
:101090008FCF81F31088654533DB0699016107998D
:1010A00041618260C0F80CE0418889B20131C1F32E
:1010B0000E0101B9012141802846FFF7C0FD2369D7
:1010C000EFF3108272B6D3E8CFCF0121BCF1000F4D
:1010D000F9D1C3E84C1FBCF1000FF4D1BFF35F8F0F
:1010E000A388F353A58021690023C1E88F3F82F3D1
:1010F0001088E368217801228A4003F501535A6081
:10110000F8BD4FF0FF30FBE770B582B006461546DC
:101110001C469DF8203033B900F0AEF9854264EBEF
:10112000010100290ADB079B0193069B00932A46D5
:1011300023463046FFF788FF02B070BD0020FBE772
:10114000F0B585B007460E4615461C46FFF768FF0A
:101150009DF828300293019400953A463346FFF7F4
:10116000D3FF05B0F0BD03464089B0EB214F31DD20
:1011700010B50A14586902EB420200EBC2001A696A
:10118000EFF3108C72B6D2E8CF4F5FF0010E002C57
:10119000F9D1C2E844EF002CF5D1BFF35F8F42884C
:1011A00092B289B28A420FD0002019690022C1E8A8
:1011B0008F2F8CF3108830B1DA681B7801219940A9
:1011C00002F50153596010BD42F4004242800120F3
:1011D0009871EAE70020704710B50446FFF720FF3A
:1011E0002146FFF7C0FF10BD40787047F0B583B0CF
:1011F000EFF30583DBB2CBB904460D46861F41F100
:10120000FF37B04271EB070301D20026374600F0EA
:1012100033F9301A67EB0103012873F1000308DA90
:101220002046294600F030F903B0F0BD1848FFF71A
:1012300051F900230093174A30463946FFF780FFE3
:10124000002819DAECE7144B1A68EFF3108172B634
:10125000D2E8CFCF0120BCF1000FF9D1C2E84C0F8A
:10126000BCF1000FF4D1BFF35F8F1A680023C2E80E
:101270008F3F81F3108820BF084B5B6A9F42E2D802
:10128000064A926AB242CBD29F42C9D1DBE700BF85
:1012900068780010450C0010C01E002000000B40B4
:1012A00038B505460C4600F0E7F8281844EB010174
:1012B000002902DBFFF79AFF38BD4FF0FF306FF0D7
:1012C0000041F7E708B5C30E4101091A63F10003B5
:1012D0009B0043EA91738900091843F10003DB0086
:1012E000C80043EA5171FFF7DBFF08BDF0B583B0DA
:1012F0000C46EFF30583DBB293B13A4B5B6A8B424A
:1013000009D3384A926A824208D2A34201D001200E
:1013100002E0002000E0002003B0F0BD0120FBE768
:101320000546FFF77DFEC3681F460678184600F0A5
:101330008DF82A1A64EB0101331D57F823301B1A6C
:101340009A4271F1000112DB20BF264B5B6A9C427E
:1013500009D8244A926AAA4207D29C4201D00120AD
:10136000DAE70020D8E70020D6E70120D4E7002301
:1013700000931D4A28462146FFF7E2FE002818DDAB
:10138000184B5B6A9C4205D8164A926AAA4202D25E
:101390009C4200D120BFFFF71FFF124B5B6A9C42AB
:1013A0001BD8104A926AAA4219D29C4213D001203B
:1013B000B2E70C4B5B6A9C4209D80A4A926AAA427D
:1013C00007D29C4201D00120A6E70020A4E700201C
:1013D000A2E70120A0E700209EE700209CE7012073
:1013E0009AE700BF00000B40450C00100048704712
:1013F00000000B4010B50A4B1B6923B10A210948B4
:10140000FFF79AFB10BDFFF7F1FF0446032100F040
:101410000BF81023032221460148FFF7C3FDEDE737
:10142000AC0E0020C01E002008B5054ADFF818C029
:10143000044B604514BF1846581CFFF77FF808BDE1
:10144000B8780010281A002000800B400246436A3A
:10145000906A1946536A9942FAD17047416A00E08E
:10146000416A9942FCD300E0416A994202D1816A03
:101470009142F9D37047000008B50248FFF7E6FF34
:1014800008BD00BF00000B4008B502460B460248ED
:10149000FFF7E4FF08BD00BF00000B4070B5154624
:1014A0001E4600EB400C4FEA8C0C0CF1804C0CF506
:1014B000803CDCF80430049A934201D2CCF804203A
:1014C000041FE4B2012C2AD90CF540534FF40062FA
:1014D0001A60204B53F820204AB15B69B3FBF2FE3F
:1014E0000EF1010E0EEB4E0EBEF1030EFCD2DCF837
:1014F000002082EA451202F0E0020CF5805ECEF890
:101500000020012C17D90CF500534FF400621A602B
:10151000049BCCF804300F4B43F8206070BD0129C8
:10152000D2D10CF5405303221A60DCF8083013F0D6
:10153000010FFAD0DBE7DCF800304B4003F0030387
:10154000CEF80030DCF8083001228A401342F9D08E
:10155000D9E700BF2C1A002000B583B04FF4803CBF
:10156000CDF800C0FFF79AFF03B000BD014B53F860
:10157000200070472C1A002038B58E469446049AF5
:101580003349B1FBFEF1334C6444334DAC4234D8A3
:10159000BCFBF1F4A4F11005B5F5987F33D85D1EBE
:1015A000062D36D8551E062D33D8B1EB1C1F36D864
:1015B000120342EA03410368002B36DB274B9842B3
:1015C00043D00E2301229A40254B1A6003F5805325
:1015D0001A60244B9B6832EA0303FAD1C0F800E09A
:1015E000846000F540520432212313600368002B0D
:1015F000FCDAC1600823136038BD1B4B1B4A112164
:101600001B4801F063FC1B4B184A1921184801F0D4
:101610005DFC194B154A1C21154801F057FC174B6E
:10162000124A2321124801F051FC036803F03F03E2
:101630007345C3D18368C3F30B03A342BED1C36810
:1016400003F4EE238B42B9D1D6E70F23BAE700BFEC
:10165000001BB70080E84BD380F8A932008005401A
:101660000020024000000240DC7800100C7F0010D7
:101670002C79001098790010B4790010007A0010CD
:10168000024B1A68024B5A60704700BF881E002048
:1016900000800D4008B5164B4FF080421A60A3F54C
:1016A0004123144A9A6051B103F540234FF0E062A0
:1016B0001A6048B9104B4FF000421A6008BD0C4B3D
:1016C0004FF0E0621A60F4E74FF47A7303FB00F026
:1016D0000A4B1860B0F1807F02D36FF07F421A602E
:1016E000FFF7CEFF044B4FF080421A60E6E700BFE1
:1016F00000B00D40F3FFFF0100A00D40881E002048
:1017000008B50E4B4FF0804CC3F800C098B140F0C4
:1017100001030B48DFF82CC0C0F81CC0DFF828C05C
:1017200083EA0C0CC0F820C041628362002110469D
:10173000FFF7B0FF08BD024BD861F7E700B00D40DE
:1017400000800D40D3C007B02D3FF84F054A00EB95
:10175000400302EB8303596000EB4000800001234B
:1017600013507047008010402DE9F04105460E46A9
:10177000174698460023DB8A002242E800F212F462
:10178000800F0BD1102144F2522098470446434663
:101790003A4631462846A047BDE8F081042144F28C
:1017A000522098470446F2E708B50023DB8A00225E
:1017B00042E800F212F4800F02D11021984708BDD0
:1017C00004219847FBE708B5031E04DB41F0200025
:1017D0003AB141F030010A460A214FF48170FFF717
:1017E000C3FF0146F7E70000034BD3F82838002B6E
:1017F000FAD0BFF35F8F704700000E40002207E071
:10180000054B13449B00BFF35F8F00211960013229
:10181000072AF5D9704700BF0382031008B5FFF708
:10182000EDFF08BD074B4FF42A621A604FF48D722A
:10183000DA6003F50053044A1A60024B5B68002B20
:10184000FBDA70470080044000B0FA0010B504468F
:1018500002E054F8043B9847014B9C42F9D310BD79
:10186000787400107047000008B50248FFF7EEFFDB
:1018700008BD00BF38740010064B074A1A6003F514
:101880008053064A1A60064B9A68044B9343FAD178
:10189000704700BF002002407F3BEFEFF6FFF303ED
:1018A00000000240054BDB6CB3F5004F00D07047E1
:1018B000034B4FF48022DA64F9E700BF00001150B7
:1018C000002011504FF0E022D2F8881D034B0B434B
:1018D000C2F8883D10EE3004704700BF03033000AB
:1018E000054B6FF060421A60044B9B68DB4333F09A
:1018F0006043F9D1704700BF003002400000024051
:1019000008B545F25320FFF74FFF034604209847E0
:1019100008BD08B545F25320FFF746FF03460120F6
:10192000984708BD08B5FEF76FFE08BD10B50C4915
:101930000C4A521A92101446442A28BF442292009C
:10194000094805F057FC04E0084A074B43F82420F7
:101950000134432CF8D9044A054B9A6010BD00BFEE
:101960000000001010010010000000201101001004
:1019700000ED00E038B50420FFF7F8FD064BA3FBAF
:101980000035AD0C002404E02946E0B2FFF7DEFE8E
:101990000134052CF8DD38BD83DE1B4330B583B040
:1019A000264B0022C3F88420FFF73CFF244B012282
:1019B000DA63224B5B6C012BFBD1214B03221A63B0
:1019C0001E4B9B6B012BFBD10224009405231D4A67
:1019D00001211D48FFF7D0FD052500952B461B4A28
:1019E00001211B48FFF7C8FD1A4B002221460420A5
:1019F000FFF7B2FD184C2346002201212846FFF7CD
:101A0000ABFD164D2B46002211460820FFF7A4FD22
:101A10002B46002211460920FFF79EFD2346002297
:101A200011460620FFF798FD2346002211460720A5
:101A3000FFF792FDFFF79EFF03B030BD00000140AD
:101A400000300140002F685900000540008C864797
:101A500000800540001BB70080D1F008006CDC025C
:101A600086B003B451FC0804CDE9020151FC09041D
:101A7000CDE9040151EC0A04CDE9060103BCF047AD
:101A8000BDE800504EEC00C4BDE800504EEC01C46F
:101A9000BDE800504EEC02C400BD000000B5FFF7E9
:101AA000DFFF02E010FE30F4F8D441EC100443EC08
:101AB000112400EE010410EE010480EE200451EC2C
:101AC0001004704700B5FFF7CBFF02E010FE30F4C2
:101AD000F8D441EC100443EC112400EE010410EEA4
:101AE000210480EE200451EC3004704700B5FFF76C
:101AF000B7FF02E010FE30F4F8D410B541EC10044A
:101B000043EC112451EC040453EC0524A0FB024CDB
:101B10005FF0000EE0FB03CEE1FB02CE4CEC204474
:101B20000024E1FB03E444EC30E480EE200451ECBB
:101B30005004BDE81040704700B5FFF791FF02E088
:101B400010FE30F4F8D441EC100443EC112451ECB5
:101B50002104A0FB01126FEA820252FB100052FB2B
:101B600012F252FB1000A0EBD07C53EC04245CFB7F
:101B700013F153EC1524A1FB022001FB030053ECED
:101B80004424A2EB000050FB1CF24FEA111312EBAD
:101B9000017043EBE27140EA515020EA915020F08D
:101BA000070053EC7524A0FB023C53EC752400FBAA
:101BB00003CC01FB02CC53EC0424ACEB824C40EA96
:101BC0005C70A0F1010041EC400480EE200451EC77
:101BD0007004704700B5FFF743FF02E010FE30F4D9
:101BE000F8D440EC700400EE010410EE210480EE05
:101BF000200451EC3004704700B5FFF731FF02E0DC
:101C000010FE30F4F8D440EC600400EE010410EE55
:101C1000210480EE200451EC3004704700B5FFF73A
:101C20001FFF02E010FE30F4F8D441EC800400EE17
:101C3000010410EE010480EE400410EE130470471E
:101C400000B5FFF70DFF02E010FE30F4F8D441ECD0
:101C5000800400EE010410EE010480EE400410EE5A
:101C60003304704700B5FFF7FBFE02E010FE30F4CE
:101C7000F8D441EC100443EC112400EE010410EE02
:101C80003004C0F30070704700B5FFF7E9FE02E0D2
:101C900010FE30F4F8D443EC102441EC110400EEB3
:101CA000010410EE30F48CBF01200020704700BF0B
:101CB00000B5FFF7D5FE02E010FE30F4F8D443EC97
:101CC000102441EC110400EE010410EE30F42CBF9E
:101CD00001200020704700BF00B5FFF7C1FE02E001
:101CE00010FE30F4F8D441EC100443EC112400EE63
:101CF000010410EE30F42CBF01200020704700BF1B
:101D000000B5FFF7ADFE02E010FE30F4F8D441EC70
:101D1000100443EC112400EE010410EE30F48CBFEB
:101D200001200020704700BF704720B108B50A6845
:101D30004968904708BD70470146002008E000EB65
:101D40008000531C0B60137803EB4003A3F13000B9
:101D50000A681378303BDBB2092BF0D970472DE9C4
:101D6000F04F83B005460E4693461F46DDF830809F
:101D70000D9CDDF838900F9B13F00202009228D1E1
:101D800013F0010F0FD05A461BE002F1010B3B4646
:101D900031462020A8470AF1010A5A46CA45F4D321
:101DA000DDF804B00DE0A2465A46CDF804B0F5E7E0
:101DB000013C02F1010A3B46314618F80400A847ED
:101DC0005246002CF4D1009B5BB9104603B0BDE82D
:101DD000F08F5A46F5E7541C3B4631462020A84771
:101DE0002246A2EB0B034B45F5D3EEE72DE9F0417C
:101DF00084B004460D4616461F46DDF828E0DDF89F
:101E00002CC09DF830301A4698460E980F99109BBA
:101E100013F0020F21D169B113F0010F0AD012B9EA
:101E200013F00C0F06D0013904E030220EF80C201C
:101E30000CF1010C844502D2BCF11F0FF5D913F04F
:101E4000010F0AD08C4508D2BCF11F0F05D83022F3
:101E50000EF80C200CF1010CF1E713F0100F17D065
:101E600013F4806F06D1BCF1000F03D0844529D054
:101E70008C4527D00D9A102A3CD00D9A022A47D0C3
:101E8000BCF11F0F0FD830220EF80C200CF1010C02
:101E9000BCF11F0F07D84246002A42D02D220EF86F
:101EA0000C200CF1010C03930291CDF804C0CDF885
:101EB00000E03B46324629462046FFF750FF04B07B
:101EC000BDE8F081BCF1010220D00D9810280FD0A0
:101ED00094460D9A102AD0D113F0200FCDD0BCF12A
:101EE0001F0FCAD858220EF80C200CF1010CC7E7BE
:101EF000ACF1020C13F0200FEBD1BCF11F0FE8D8AE
:101F000078220EF80C200CF1010CB9E79446B1E7E9
:101F1000BCF11F0FC7D862220EF80C200CF1010C87
:101F2000AEE713F0040F05D02B220EF80C200CF1B5
:101F3000010CB8E713F0080FB5D020220EF80C20E2
:101F40000CF1010CAFE7F0B591B00D4616461F46F7
:101F5000169B189A1B990BB921F0100111F4806E91
:101F60001DD063B34FF0000E19E011F0200F24D004
:101F70004124A4445FFA8CFCACF10A0C5FFA8CFC9F
:101F80000EF101040EF1400EEE440EF820CCB3FB2E
:101F9000F2FC934214D31F2C12D8A6466346B3FB1F
:101FA000F2FC02FB1C3C5FFA8CFCBCF1090FDCD894
:101FB0000CF1300C5FFA8CFCE2E76124D9E71C4697
:101FC00006911A9B0593199B049303929DF85C302C
:101FD0000293019408AB00933B4632462946FFF733
:101FE00005FF11B0F0BD2DE9F04F95B08346099182
:101FF0000A920B931E9F1F9DDDF88880DDF88C9060
:10200000DDF898A057EA050301D12AF0100A1AF466
:10201000806422D057EA05032DD000241DE01AF079
:10202000200F26D041231344DBB20A3BDBB2661CEF
:1020300004F150020DEB020404F8203C42464B46EA
:102040003846294605F0D4F9474575EB090513D301
:102050001F2E11D8344607460D4642464B46384699
:10206000294605F0C5F9D2B2092AD8D83032D3B200
:10207000DDE76123D7E70026CDF818A0259B05935F
:10208000249B0493CDF80C809DF880300293019638
:102090000CAB00930B9B0A9A09995846FFF7A6FED2
:1020A00015B0BDE8F08F00002DE9F04F93B0044665
:1020B0000D460E921E46DDE91C8942464B464046BF
:1020C0004946FFF7D3FD002840F0FE804FF0FF3275
:1020D000B54B40464946FFF717FE002840F0F48014
:1020E0004FF0FF326FF4801340464946FFF7D0FDB2
:1020F000002840F0E9800022002340464946FFF7CF
:10210000C7FD002840F0F180CDE90689209B13F43B
:1021100080630F9301D106231E93DDE906AB52467F
:102120005B46CDE90A23079B5AEA030100F0E780EA
:10213000C3F30A50C3F313034FF0000A4FF0000B30
:10214000CDE908AB089243F07F53099343F4401361
:102150000993A0F2FF30FFF741FD81A3D3E90023EB
:10216000FFF7C8FC80A3D3E90023FFF79BFC82465E
:102170008B4600228D4BDDE90801FFF7A7FC7CA30D
:10218000D3E90023FFF7B6FC02460B4650465946FA
:10219000FFF788FCFFF746FD0890FFF71FFD82461A
:1021A0008B4675A3D3E90023FFF7A4FC0022804BE4
:1021B000FFF778FCFFF736FD074671A3D3E900234C
:1021C00050465946FFF796FC82468B463846FFF745
:1021D00005FD6DA3D3E90023FFF78CFC02460B46F7
:1021E00050465946FFF772FC02460B4682468B4624
:1021F000FFF780FCCDE90C0107F2FF33002100223C
:10220000CDE90A121B050B9300230A935046594649
:1022100052465B46FFF746FCCDE9100152465B464D
:1022200000204FF08041FFF751FC82468B46002290
:10223000604BDDE90C01FFF783FC00225E4BFFF7EA
:1022400031FC02460B46DDE90C01FFF779FC002268
:102250005A4BFFF727FC02460B46DDE90C01FFF75E
:102260006FFC02460B4650465946FFF71BFC0246E0
:102270000B46DDE91001FFF763FC0022504BFFF72E
:1022800011FCDDE90A23FFF735FC02460B46CDE9D8
:102290000C23DDE90CABCDE90AABDDE90623FFF742
:1022A00033FD50B1089B013B08930022424BDDE90E
:1022B0000C01FFF745FCCDE90A01089B6333C62BEF
:1022C00048D804231F461EE0209B04931F9B0393C2
:1022D0001E9B0293CDE9008933460E9A294620467B
:1022E00000F002F913B0BDE8F08F9FED297B8DED72
:1022F000067BCDF8188009F10043079306E7002319
:10230000089304231F46209B13F4006F63D0DDE97C
:102310000A1213460B4315D01FA3D3E90023DDE9AE
:1023200006AB50465946FFF7DBFC002800F0B680AC
:102330001BA3D3E9002350465946FFF7A9FC002808
:1023400000F0AC801E9A089B9A423BDDD31A013BF9
:102350001E9339E005231F46D5E700BFAFF3008089
:10236000FB799F501344D33FB3C8608B288AC63F84
:1023700061436F63A787D23F71A379094F930A40E6
:102380001655B5BBB16B0240EF39FAFE422EE63F5F
:1023900000000000000000002D431CEBE2361A3F55
:1023A0000000000080842E41FFFFEF7F0000F83F17
:1023B0000000E03F00002C400000244000001840D6
:1023C0000000F03F00231E93209B43F48063209382
:1023D00000231F4608931F9A974269D2D31B9A463F
:1023E000209B13F002039B4602D00FB100239A46B4
:1023F000089B3BB1DDE90A23DDE90601FFF7A0FBFD
:10240000CDE906010022002340464946FFF740FC83
:10241000002850D1209B23F400630493CDF80CA036
:102420001E9B02939DED067B8DED007B33460E9A3D
:102430002946204600F058F8002F3FF453AF209B68
:1024400013F0200F3FD04FF0450C00F10108334648
:10245000024629466046A047089981EAE172A2EB4C
:10246000E172052305937B1E0493002303930A2343
:102470000293CB0F019300923346424629462046F1
:10248000FFF761FD5B46002B3FF42CAF0246DDF801
:10249000389037462E4625461F9C1EE01E9B002B7B
:1024A00099D00F9B002B96D01E9B013B1E9392E769
:1024B00000239A4694E7DDE90601024601F1004354
:1024C000CDE90623A6E74FF0650CBEE702F101084F
:1024D0003B4631462020A8474246A2EB0903A342CF
:1024E000F4D31046FEE600BF2DE9F04F2DED028B30
:1024F00095B00790089109920A93DDE92089229D01
:1025000042464B4640464946FFF7B0FB002834D1CF
:102510004FF0FF326FF4801340464946FFF7B8FB97
:10252000002839D14FF0FF32A94B40464946FFF70A
:10253000EBFB00283FD1A2A3D3E900234046494644
:10254000FFF7E2FB00284CD19FA3D3E900234046CC
:102550004946FFF79DFB002843D100220023404657
:102560004946FFF795FB002849D10B90249B13F4B3
:10257000806F00F0B580002454E0249B0393239BDC
:10258000029303230193934B00930A9B099A0899A2
:102590000798FFF7E4FB50E1249B0393239B0293EE
:1025A000042301938C4B00930A9B099A089907987E
:1025B000FFF7D5FB41E1249B13F0040F0ED0874BAE
:1025C00004222499039123990291019200930A9B7A
:1025D000099A08990798FFF7C2FB2EE1804B032266
:1025E000EFE7249B0493239B03930295CDE9008995
:1025F0000A9B099A08990798FFF756FD1DE1424684
:102600004B4600200021FFF761FA804689460123EE
:102610000B93ABE704F150036B44302203F8202CFA
:10262000013D01341F2C01D8092DF3D840464946FD
:10263000FFF7F8FA0646FFF7D1FA02460B46404686
:102640004946FFF743FA674B03EBC50393ED007B65
:10265000B0EE478AF0EE678A53EC172BFFF74AFA81
:1026600082468B46FFF7F0FA0746FFF7C9FA0246A3
:102670000B4650465946FFF729FA82468B46002200
:10268000594BFFF741FB68B301373846FFF7B8FAFB
:1026900002460B4651EC180BFFF70EFB08B1013652
:1026A00000276DBB3046FFF799FA02460B464046BD
:1026B0004946FFF70BFA8046894600224A4BFFF74E
:1026C000E7FA00284CD10022474B40464946FFF725
:1026D0001BFB002844D116F0010F41D001363FE02A
:1026E000062548E70022404B50465946FFF7D0FAEE
:1026F0000028D6D117B117F0010FD2D00137D0E79B
:102700001F2C17D8013D394BA3FB0723DB081946C3
:1027100003EB8303A7EB4303621C303304F1500047
:102720000DEB000404F8203C092F02D90F46144693
:10273000E6E714461F2C0AD86B1E45B104F150027F
:102740006A44302102F8201C1D460134F2E71F2C98
:1027500006D804F150036B442E2203F8202C0134D8
:102760001F2C17D8224A82FB0632F317C3EBA203B1
:102770001A4603EB8303A6EB4303611C303304F1D9
:1027800050000DEB000404F8203C16460AB10C463C
:10279000E6E70C46249B13F0020F36D113F0010F2D
:1027A00033D0239B002B4DD00B9B1BB9249B13F0E4
:1027B0000C0F49D0239B013B2393194621E000BF16
:1027C0000000000065CDCD410000000065CDCDC109
:1027D000FFFFEF7F687A00106C7A00105C7A0010BF
:1027E000647A0010707F00100000E03FCDCCCCCCAC
:1027F0006766666604F150036B44302203F8202CB0
:1028000001348C4201D21F2CF4D91F2C08D80B9B09
:10281000E3B104F150036B442D2203F8202C013462
:10282000249B0393239B029301940CAB00930A9B7C
:10283000099A08990798FFF792FA15B0BDEC028B38
:10284000BDE8F08F2399DCE72399DAE7249B13F0A6
:10285000040F07D004F150036B442B2203F8202C03
:102860000134DDE7249B13F0080FD9D004F15003A5
:102870006B44202203F8202C0134D1E72DE9F04FDE
:102880008FB0804617460D938946002900F0F682E6
:1028900000260D9B1878002800F0F382252809D027
:1028A000741C3B4632464946C0470D9B01330D938D
:1028B0002646EEE701330D93002511E0202A24D0AF
:1028C000232A05D145F0100501330D93012306E0BD
:1028D000002304E045F0020501330D930123E3B129
:1028E0000D9B1A782B2A0AD0E8D92D2AF2D0302A4B
:1028F00011D145F0010501330D930123EFE745F0B8
:10290000040501330D930123E9E745F00805013380
:102910000D930123E3E70023E1E70A930D9B1A7867
:10292000A2F13003DBB2092B15D92A2A18D0DDF821
:1029300028B00D9B1A782E2A22D00D9B1A786C2A6B
:1029400043D039D9742A5CD07A2A5ED145F4807597
:1029500001330D9359E00DA8FFF7EEF98346E8E740
:10296000189B1A1D18921B68002B04DB9B460D9BBD
:1029700001330D93DDE745F00205C3F1000BF6E7E7
:1029800045F480655A1C0D925A78A2F13003DBB2EF
:10299000092B0CD92A2AD0D1189B1A1D18921C6811
:1029A00024EAE4730A930D9B01330D93C5E70DA848
:1029B000FFF7C2F90A90C0E7682A14D06A2A24D126
:1029C00045F4007501330D931FE045F480715A1CE6
:1029D0000D925A786C2A01D00D4616E045F44075E8
:1029E00002330D9311E045F080015A1C0D925A7884
:1029F000682A01D00D4608E045F0C00502330D936A
:102A000003E045F4807501330D930D9B187865281C
:102A10003DD071D8462800F0878018D963282FD17F
:102A200015F0020500F0A48101241898031D1893E5
:102A300006F1010A3B46324649460078C047002D60
:102A400040F099810D9B01330D93564621E72528CF
:102A50000AD1741C3B46324649462520C0470D9B8F
:102A600001330D93264614E7452810D0741C3B46CD
:102A700032464946C0470D9B01330D93264608E771
:102A80002CD858282CD062282AD04728EED1672885
:102A900001D0472801D145F40065452801D04728D9
:102AA00001D145F02005189B073323F0070303F1FC
:102AB000080218920495CDF80CB00A9A0292D3E954
:102AC0000023CDE900233B46324649464046FFF706
:102AD000EBFA06460D9B01330D93DAE66428C5D167
:102AE00078284BD058287CD06F287CD062287CD0A6
:102AF00025F010050A2342E0702800F0A4810ED9C9
:102B0000732834D1189B1A1D1892D3F800A00A9B81
:102B1000002B40F05A814FF0FF3253463BE16728CB
:102B2000B5D01FD86628A1D1462800F01181189B86
:102B3000073323F0070303F1080218920495CDF838
:102B40000CB00A9A0292D3E90023CDE900233B4658
:102B5000324649464046FFF7C7FC06460D9B013307
:102B60000D9396E66928BBD06F28B9D07EE7FFF4B5
:102B70007DAF7528B4D07828B2D077E710235828D5
:102B800035D0692803D0642801D025F00C0515F450
:102B9000806F01D025F0010569282BD0642829D049
:102BA00015F4007F40F0968015F4807F40F0AE80F1
:102BB00015F0400F00F0BF80189A111D189112787F
:102BC0000595CDF810B00A99039102930023019363
:102BD00000923B46324649464046FFF7B4F9064666
:102BE00029E01023CBE70823C9E70223C7E745F014
:102BF0002005C6E715F4007F21D115F4807F42D16E
:102C000015F0400F58D0189A111D1891127882EAC9
:102C1000E271A1EBE2710595CDF810B00A9803902E
:102C20000293D20F019200913B46324649464046FC
:102C3000FFF789F906460D9B01330D9329E6189A93
:102C4000073222F0070202F1080118915168126858
:102C50000846002913DB0895CDF81CB00A9C0694A1
:102C6000049300230593C90F0291009201903B4603
:102C7000324649464046FFF7B6F90646DBE7524280
:102C800061EB4100E7E7189A111D1891126882EA7A
:102C9000E271A1EBE2710595CDF810B00A980390AE
:102CA0000293D20F019200913B463246494640467C
:102CB000FFF749F90646BEE715F0800F05D0189AD0
:102CC000111D1891B2F90020A1E7189A111D189151
:102CD00012689CE7189A073222F0070202F10801F5
:102CE00018910895CDF81CB00A990691002104931B
:102CF00005910291D2E90023CDE900233B463246FB
:102D000049464046FFF76FF9064694E7189A111DA9
:102D100018910595CDF810B00A99039102930023FC
:102D20000193136800933B46324649464046FFF7FD
:102D30000AF906467FE715F0800F04D0189A111D96
:102D4000189112883CE7189A111D1891126837E7FC
:102D500045F02005EBE602F1010A3B4649462020FA
:102D6000C047234652465C1C9B45F4D816465CE699
:102D700001233246F7E7524606E0561C3B464946D9
:102D80002020C0472C463246651CA345F5D8924604
:102D900058E601330A46197811B1511E002AF8D1BC
:102DA000A3EB0A0315F480620B9203D00A9A9342B4
:102DB00028BF134615F0020409D032460B9E0B942F
:102DC000CDF830B00A9D9B461FE00A9AA5E6324630
:102DD000264606E0541C3B4649462020C0472B4669
:102DE00022465D1C9B45F5D834462B460B9E0B9422
:102DF000CDF830B00A9D9B4607E01D460AF1010A56
:102E0000541C3B464946C04722469AF8000020B170
:102E1000002EF3D06B1E002DEFD116460B9C5B46A7
:102E2000DDF830B054B90D9B01330D9331E5551CDD
:102E30003B4649462020C04723462A465C1C9B450A
:102E4000F5D81646EFE745F02105189B1A1D189294
:102E50001B680595082204920A9A03921022029296
:102E60000022019200933B46324649464046FFF716
:102E70006AF806460D9B01330D930AE5DFF81C80C6
:102E800006E5BE4208D37A1E3B4649460020C047AD
:102E900030460FB0BDE8F08F3246F5E7291D00102F
:102EA00000B585B002900391009313464FF0FF32B6
:102EB00002A90248FFF7E2FC05B000BD2B1D00107F
:102EC00000BEFDE708B5FFF7FBFF000000B583B0CB
:102ED0008C46194662B19646074BCDF804E0009344
:102EE00063460246054800F051F90120FFF7E8FF6C
:102EF000034B9E46F1E700BF747A0010847A0010FD
:102F0000807A001010B5EFF30583DBB203B100BE89
:102F1000FEF7AAFC044C02E054F8043B9847034B2C
:102F20009C42F9D310BD00BF787400108474001067
:102F300008B5034608461B681146984708BD0000BF
:102F4000F8B507460D461646437D13B100242046CA
:102F50000CE003681146284698472CE03B7D0FE0C3
:102F60003B68022114489847601C0134B44213DACC
:102F7000002CF3DD631EEB5C0D2B14BF002301233B
:102F80002A5D0A2AF1D1002BEFD1A042E8DA3B6892
:102F9000211A28449847E3E7B04203DA3B68311A24
:102FA00028449847002E06DD013EAB5D0D2B14BF73
:102FB000002301233B75F8BDC07F001038B50368BE
:102FC000B3B105460B4B1C6806E0294651F8042BAB
:102FD0002046FFF7B5FF24694CB12368002BFAD0D7
:102FE000054B1B68002BF0D0A342F4D1EDE72C6019
:102FF00038BD00BF7C1A0020841A002038B5054671
:103000000C460B68802B05D023685A1C22601C4498
:10301000257138BD0846FFF7D1FFF5E708B5FEF783
:103020002BFA074A821841F10003002B03DB054805
:1030300004F0EEF908BD4FF0FF326FF00043F6E701
:1030400040420F00000F002008B5024804F0D4F9F8
:1030500008BD00BF000F00202DE9F04383B00646F5
:103060000D4690461C46FFF7D9FF8146B5F1FF3F5C
:1030700004D044B1164F174B1C6807E0304604F0EB
:103080002FF90546F5E7144FF5E72469BCB123682D
:10309000002BFAD0114B1B680BB1A342F5D12A4685
:1030A00031462046B847B8F1000FEED00A238DF81C
:1030B000073001220DF107012046B847E5E74B46EE
:1030C0001BB9284603B0BDE8F083FFF7BDFFF8E762
:1030D000412F00107C1A0020312F0010841A00208C
:1030E000084A136802E003F110021B693BB1136840
:1030F0008342F8D129B9036913600161704701B1B6
:10310000106070477C1A002010B5054B1C6800E069
:10311000246924B16368002BFAD09847F8E710BD02
:103120007C1A002008B500F0B7F908BD38B505468F
:1031300004F0D6F8044601231A4601462846FFF754
:103140008BFFFFF7E1FF204638BD0000F0B5A3B0CC
:1031500007460E46FFF762FF05460023019301ACC8
:1031600033463A4621460848FFF79AFE064620466F
:10317000FFF724FFFFF7C8FF15B9304623B0F0BDB5
:10318000FFF762FFF9E700BFFD2F00100FB400B595
:1031900083B004A951F8040B0191FFF7D7FF03B0E6
:1031A0005DF804EB04B0704770470000014B00224B
:1031B0001A707047E11E00204B79FF2B0BD18B79E1
:1031C0005BB9CB79012B0AD1082A0AD98A78064B38
:1031D0001A700920704700207047002070470020B7
:1031E00070470020704700BFE11E0020012070479B
:1031F000012923D108B59188114B1B78994201D040
:10320000002008BD5378012B03D0022B0FD00020E3
:10321000F7E7518811F4807F06D0480AC1F34022B5
:1032200001F07F01FEF7CFFA4FF0FF30F6E764229E
:1032300000210846FEF764FA0120E2E7012070470A
:10324000E11E0020004870478C80001001290FD13A
:1032500008B594465378012B0CD19388072B01D0E5
:10326000002008E0A623044A614601F03BFC02E08E
:1032700001207047002008BDE47F00100123037087
:1032800000487047C47F001008B50B68B3F5966F0F
:1032900000D008BD002211464FF0FF30FEF793FA30
:1032A000024B1860024B1960704700BF1C1A0020C7
:1032B000201A002008B5FEF7DFF80E4A821841F107
:1032C0000003002B11DB0C4804F0A2F860B10021D0
:1032D0004FF0FF3001F090FA002001F08FFD002840
:1032E000F5D1054804F088F808BD4FF0FF326FF0C3
:1032F0000043E8E740420F00C41E002038B51B4BD6
:103300001B68002B27D0EFF3108272B6D3E8CF0FE3
:1033100001210028FAD1C3E8401F0028F6D1BFF3ED
:103320005F8F12494A600023114803700968C1E8A1
:103330008F3F82F310880022002314461D460D4B58
:103340001878FDF7D1F960B90022002314461D4614
:103350002046294638BD4FF47A72002314461D4694
:10336000EDE7044B1878FDF7E9F9F1E7901E00202E
:10337000E31E0020E21E002008B5024B1878FDF77E
:10338000DDF908BDE21E002070B584B00646154682
:103390001C46FEF771F82A1844EB0103002B0BDBE7
:1033A0009DF82810029109990191089900913046E1
:1033B000FDF7AAFE04B070BD4FF0FF326FF000437E
:1033C000EEE7F0B585B007460E4615461C46FDF7FC
:1033D00027FE9DF828300293019400953A46334623
:1033E000FFF7D2FF05B0F0BD10B582B00021244830
:1033F00004F016F8002822D1224B1B68EBB1EFF342
:10340000108272B6D3E8CF0F01210028FAD1C3E8A9
:10341000401F0028F6D1BFF35F8F1A494A601A484F
:103420000378DBB24FF0010C80F800C0086800217F
:10343000C0E88F1F82F31088BBB102B010BD00211D
:103440004FF0FF3001F0D8F9002001F0B1FC044644
:103450000B4803F0D1FF002CEFD00C4B1B68002B66
:10346000EBD00B4A10689847E7E7CDF800C00B4651
:10347000084A4FF47A700021FFF7A3FFDDE700BF91
:10348000C41E0020901E0020E31E00201C1A0020F5
:10349000201A0020FD32001010B582B04FF05043CA
:1034A0001C68FDF7BDFDFDF79FFEA0422DD1244B0A
:1034B0001B780021084602F045F9224B1B6853B3E4
:1034C0000120FDF725FBC0B21F4C20701F49FDF7FE
:1034D00055F901212078FDF727F90E20FDF742F973
:1034E0000446E0B10120FDF777F801461848FDF7E2
:1034F0006BFB002217490E20FDF770F901211648D9
:10350000FFF7EEFD204602B010BD144B144AC62151
:103510001448FFF7DBFC0B48FDF714FBD0E70C4A1F
:10352000034610605060012200920F4A4FF47A70F7
:103530000021FFF746FFC443E40F002CE2D0DDE793
:103540003CA30010C41E0020E21E0020E93300103E
:10355000901E002079330010C40E0020B47A0010B1
:10356000BC800010BC7A0010FD32001008B50020AD
:1035700001F004FC08BD000038B504460D46FFF715
:10358000F5FFA0B3002001F013FCA0B3FDF774FF1A
:103590001D4A821841F10003002B17DB1B4803F082
:1035A00037FF60B3FFF7E2FF18B1002001F000FC25
:1035B00088B901464FF0FF3001F01EF96FF00203A9
:1035C0001C46124803F018FF204638BD4FF0FF326A
:1035D0006FF00043E2E72A462146002001F0F4FBA9
:1035E00004460028EDD16FF002031C46E9E76FF0B6
:1035F00002031C46E8E76FF002031C46E4E76FF0A5
:1036000002031C46E0E700BF40420F00C41E00203A
:10361000F8B507460D46FDF72FFF2E4A821841F1F7
:103620000003002B04DB2C4803F0F2FE28B9F8BDA0
:103630004FF0FF326FF00043F5E7FFF797FF0028E8
:1036400045D1264B00200021C3E90001224803F0A8
:10365000D3FEECE701464FF0FF3001F0CDF800203B
:1036600001F0CCFBFFF782FF0028EFD0002001F033
:1036700043FCF8B1AC42E9DA2E1B002001F03CFC1F
:10368000864200DC30460028E4D00246391900208A
:1036900001F010FC064600214FF0FF3001F0ACF8BD
:1036A000002001F0ABFB3444FDF7E6FE0B4BC3E911
:1036B0000001DFE7FDF7E0FE084A13685268084E94
:1036C0009B1942F1000283428A41D3D2BEE7002413
:1036D000D0E700BF40420F00C41E00208810002029
:1036E00020A107000048704738810010004870474B
:1036F000E480001010B50446144B1B786BB18CB9F4
:10370000134B40F209425A80012301335B009BB204
:103710000F4843F44073038010BD11210B4800F0A3
:1037200045F8ECE7052C0ED80A4B53F8240000238B
:10373000122BEAD8C25C002AE7D00133044921F8F1
:103740001320DBB2F4E70020E6E700BFCC1E002028
:10375000541A0020CC80001000B58BB045F24730E1
:10376000FEF722F803460122092101A89847042800
:1037700001D100230EE0094B094A2F210948FFF728
:10378000A5FBC3F10F0228326A4412F8241C064A32
:10379000D1540133072BF4DD0BB000BD707B00105A
:1037A0006C810010787B0010B81E002008B511B1A4
:1037B0008C46002208E0104B104A3B211048FFF7CE
:1037C00085FB3733835401320CF1FF3393420FD919
:1037D0000F2A0DD853080B49CB5CD14301F00101EE
:1037E00089000B4103F00F03092BEADC3033E9E7D2
:1037F0000023835408BD00BFEC7B00104C810010F7
:10380000787B0010B81E002000B500F07F0C4FEA56
:103810004C0E0EEBD01E2A4B03EB4E139870C009D2
:103820000CBF4FF0010E4FF0000E83F801E04FF097
:10383000000E83F803E01983DA76F0B94FEACC037F
:10384000204A1A4400EB4C011D4B03EB41139A60D4
:1038500000EB4C021A4B03EB42139B6800221A60E8
:10386000BCF1000F13D100EB4C00154B03EB4010E3
:10387000C0F804C0144BC36000BD144A02EBCC0274
:1038800000EB4C010E4B03EB41139A60E0E758B993
:103890000CF1FF33DB000E4A1A4400EB4C00084BDE
:1038A00003EB40135A60E7E70CF1FF33094A02EBE0
:1038B000C30200EB4C00024B03EB40104260DBE71D
:1038C000881A002084001050000110508000105011
:1038D0000C0010500800105008B5038B3F339B09B3
:1038E0009901C27E022A08D0084A1368C3600B44BB
:1038F0001360074A934202D808BDD901F4E7054B8B
:10390000054A52210548FFF7E1FA00BF8C1E00204E
:10391000FF0F1050F47B0010B8810010387C0010AD
:1039200070B500F07F044FEA440C0CEBD013DFF8C5
:1039300034C00CEB43131E46FFF766FF04B970BD9D
:10394000318B3046FFF7C8FFF27EF36883F0A04367
:1039500083F4801343EA826343F000437268136088
:10396000EDE700BF881A002008B500F07F035B0078
:1039700003EBD010024B03EB401000F01DF908BD23
:10398000881A002008B520B901210E20FCF7CCFED2
:1039900008BD034B034A40F297110348FFF796FA1C
:1039A000D07C0010A8810010387C001008B528B920
:1039B000024601468020FFF7D7FF08BD034B044AAB
:1039C00040F2A1110348FFF781FA00BFD07C00103C
:1039D00098810010387C0010024B4FF48032DA647A
:1039E000704700BF0020115070B548BB064600F07C
:1039F000C3F8174C0C23A367FF2216490E20FCF7CF
:103A0000EDFE40252A460021134803F097FB0022D3
:103A100029461046FFF784FF002229468020FFF741
:103A20007FFF03F001FD012525644FF00053E3649F
:103A30000A4BC4F890303046FFF7CEFF284670BDE1
:103A4000074B084A40F263110748FFF73FFA00BFEF
:103A5000000011509D030020881A002010D00100A2
:103A6000D07C0010CC810010387C0010044B197001
:103A700021B1044B4FF40032C3F89020704700BFCF
:103A8000DE1E0020002011500B7813F01F0F05D10F
:103A900013F0600F02D14B78052B00D070474B8894
:103AA000DBB2014A1360F9E700001150CA7802F056
:103AB0000302012A09D008B50B468988C1F30A011F
:103AC0009878FFF72DFF012008BD0020704708B54A
:103AD00003F0AAFC08BD000008B530B9084611463D
:103AE0001A46FFF741FF012008BD034B034A4FF47C
:103AF00001710348FFF7EAF9D07C001088810010BB
:103B0000387C001008B511F07F0304D1CA090ED12A
:103B10000220084A90665B0003EBD1134FF4006269
:103B20000021054800EB431003F06EFC08BD0120A6
:103B3000EFE700BF00201150881A002008B511F0EF
:103B40007F0300D108BD5B0003EBD113044800EBF9
:103B500043100022C2706FF4006103F055FCF1E7DE
:103B6000881A002004E011F8012B00F8012B1A46F6
:103B7000531E002AF7D1704708B54FF080530A4A08
:103B8000136002F580521360084B9B6813F0805F4E
:103B9000FAD04FF480520021054803F0CFFA054BCC
:103BA00009225A6708BD00BF002002400000024001
:103BB000000010500000115070B504460D46164626
:103BC000837EABB9A6820023E3820123A37625611D
:103BD000204603F015FC20B10B4B4FF40032C3F824
:103BE0009020204603F018FC50B10123237770BDCC
:103BF00081780648FFF7CAFA204603F0EDFBE1E7BB
:103C0000204603F0F1FBF2E700201150E87D0010A0
:103C100038B50546002408E0D21A1B4B03EB4213CB
:103C2000DB68284698470134E4B2184B1B782246DB
:103C3000591CA14215DBA342EED9154B1B6813EBAF
:103C40004413EDD140F2252212491348FFF79EFAA2
:103C50004FF0E023D3F8F03D13F0010F13D000BE76
:103C600011E00E4C54220021204603F067FA4FF079
:103C7000FF336360A360E36023612022FF2104F12E
:103C8000140003F05BFA38BDA0820010DD1E002096
:103C9000441200206C820010207E001014140020BA
:103CA00008B5FFF7B5FF00F075FF08BD70B5064613
:103CB0000C461546486900F077FF63692A460121E2
:103CC0003046984770BD00002DE9F04F83B0824622
:103CD000481EC0B2FFF70AFD20B183464378019326
:103CE000022B11D040F2D63262496348FFF74EFAF8
:103CF0004FF0E023D3F8F03D13F0010F00D000BEE9
:103D0000002003B0BDE8F08FC279C2F340105B4BD6
:103D1000197860F304111970C2F38012C9B262F30A
:103D2000451119700BF10908BBF802309B447BE088
:103D300098F8033098F8002090447DE040F2F1328A
:103D40004C494D48FFF722FA4FF0E023D3F8F03DFD
:103D500013F0010F00D000BE0020D2E7F31A484A4A
:103D600002EB4319D9F810302A464146504698478D
:103D7000082801D985421ED20134E4B2414B1B7898
:103D800026465A1CA2424ADBA342E7D93E4B1B6897
:103D900013EB4419E6D140F2FA3236493648FFF7C0
:103DA000F5F94FF0E023D3F8F03D13F0010F00D008
:103DB00000BE0020A5E73B464F468146012B11D0AF
:103DC00000218B4224D998F802200A44D2B22B4811
:103DD00010440079FF280BD12848024414710131A6
:103DE000C9B2EEE73969294A9142E9D1019BE7E777
:103DF00040F219421F492048FFF7C8F94FF0E0236D
:103E0000D3F8F03D13F0010F00D000BE002078E79A
:103E100023464A4641461E4801F0AAFDC844194BB4
:103E20001B7801339E4212DCD84520D298F801302D
:103E30000B2B3FF47DAF012398F80120042A7FF477
:103E40007DAFABEB0805ADB200241F4696E74FF4FB
:103E5000856208490848FFF799F94FF0E023D3F845
:103E6000F03D13F0010F00D000BE002049E7012013
:103E700047E700BF40820010207E0010141400208D
:103E8000A0820010DD1E00204412002065500010AA
:103E900028140020704770470020704700207047AA
:103EA00038B505460C464B881A0A062A61D01146D9
:103EB000D8B211D8022A2FD0032A4ED0012A09D114
:103EC000FFF710FC0246B8B112232146284600F045
:103ED00009FE2CE000202AE0072A1DD00F2A09D174
:103EE000FFF7B0F9024610B343882146284600F098
:103EF000F9FD1CE000201AE040F23A422249234832
:103F0000FFF744F94FF0E023D3F8F03D13F0010F31
:103F100000D000BE00200AE0022909D0FFF7BEFF52
:103F2000024620B153882146284600F0DBFD38BD0B
:103F3000FFF7DCFB02460028F4D140F2614212494F
:103F40001248FFF723F94FF0E023D3F8F03D13F0C8
:103F5000010F00D000BE0020E9E7A188FFF7CAFBEF
:103F600002460028E3D003782146284600F0BAFD37
:103F7000DDE7FFF791FF02460028D8D003782146FD
:103F8000284600F0AFFDD2E728820010207E001006
:103F90007047704770477047024B5878003818BF19
:103FA0000120704714140020024B1878C0F38000E1
:103FB000704700BF14140020024B1878FF3818BF58
:103FC00001207047F80E0020F8B506460C460F4653
:103FD000FFF7F2FF0546002854D104B35422002114
:103FE000374803F0ABF8374B00221A70364C2046A6
:103FF000FCF7A8FD354B1C60354C2046FCF7ECFD6A
:10400000143C204602F07CF8324B1C60324B23B14A
:104010003248FFF733F9324B1860002417E04FF4B1
:10402000E97230493048FFF7B1F84FF0E023D3F898
:10403000F03D13F0010F25D000BE23E0D21A2B4B28
:1040400003EB42135B687BB198470134E4B2234B26
:104050001B782246591CA14216DBA342EED9204B05
:104060001B6813EB4413EDD14FF4F8721D491E4841
:10407000FFF78CF84FF0E023D3F8F03D13F0010F79
:1040800000D000BE2846F8BD194B1E703946304698
:10409000FFF7AAFC054618B13046FFF773FCF1E7BD
:1040A0004FF4FC720F491048FFF770F84FF0E0230F
:1040B000D3F8F03D13F0010FE4D000BEE2E700BFFB
:1040C00014140020DF1E00200C14002068140020AF
:1040D000F00E00206C1400207D320010DD1E002048
:1040E0004412002090820010207E0010A082001058
:1040F000F80E002070B51B4B1B781E468B7813F012
:10410000700F0ED10C46184B9978204601F0C0FB79
:104110000546B8B121463046FFF7C8FC054628469B
:1041200070BD40F20B5211491148FFF72FF84FF0C4
:10413000E023D3F8F03D13F0010F00D000BE0023C0
:104140001D46ECE740F20C5208490948FFF71EF8FB
:104150004FF0E023D3F8F03D13F0010FDFD000BEA5
:10416000DDE700BFF80E002014140020F8810010D5
:10417000207E00102DE9F04780460C4616461F466B
:10418000DDF82090002526E040F2E7421F49204854
:10419000FEF7FCFF4FF0E023D3F8F03D13F0010FE2
:1041A00000D000BE4FF0000A5046BDE8F0874FF443
:1041B0009D6216491648FEF7E9FF4FF0E023D3F859
:1041C000F03D13F0010FEFD000BEEDE7099A137038
:1041D00023781C440135AE4214DD6378052BD3D11E
:1041E000E17801F00301B942CED121464046FFF704
:1041F00081FF82460028DAD0A378DA09E6D189F86F
:104200000030E5E74FF0010ACEE700BF088200105A
:10421000207E001008B501F07F00400000EBD110B7
:104220003030044B1844044B1968043001F0E2FAB2
:1042300008BD00BF141400206814002008B501F068
:104240007F00400000EBD1103030044B1844044B89
:104250001968043001F0F9FA08BD00BF14140020F9
:104260006814002038B52448007801F07F04DFF896
:104270008CC00CEB440C0CEBD11C0CF1300C9CF8FA
:1042800004C01CF0010F27D1CD09DFF870C00CEB82
:10429000440CAC449CF834E04EF0010E8CF834E051
:1042A000FFF71AFC38BB154B03EB44032B4493F880
:1042B000342022F0010283F8342093F8342022F0D5
:1042C000040283F834204FF0E023D3F8F03D13F0DC
:1042D000010F10D000BE0EE040F2395208490948E3
:1042E000FEF754FF4FF0E023D3F8F03D13F0010F39
:1042F00000D000BE002038BDF80E002014140020AD
:10430000E8810010207E001038B501F07F05CC094F
:104310000A4B1878FFF7F6FB094B03EB45032344E0
:1043200093F8342042F0020283F8342093F83420CA
:1043300042F0010283F8342038BD00BFF80E00209F
:104340001414002038B501F07F05CC090A4B187809
:10435000FFF7F4FB094B03EB4503234493F83420A8
:1043600022F0020283F8342093F8342022F0010274
:1043700083F8342038BD00BFF80E0020141400204C
:1043800001F07F02044B03EB420303EBD11191F8E0
:104390003400C0F340007047141400202DE9F041B0
:1043A00082B007460C46002000F0FEFB237803F0A5
:1043B0006003602B32D0402B44D0227802F01F02E1
:1043C000012A00F01281022A00F05681002A40F0F2
:1043D000E781202B40D0002B61D16378052B76D06C
:1043E00068D8012B00F0E380032B00F0CE80002B77
:1043F00040F0EF80B24B1A78930803F00203C2F347
:1044000040121343ADF8063002230DF10602214697
:10441000384600F067FB01231D460FE04FF435726C
:10442000A849A948FEF7B2FE4FF0E023D3F8F03DCB
:1044300013F0010F00D000BE00231D46284602B035
:10444000BDE8F081A14800F0AFFB224601213846CB
:10445000FEF7FCFE0546F1E7A388DAB20F2A00F268
:10446000AA81974A52FA83F31B79994A12789342A8
:1044700007D2984A116811EB43110AD100231D4657
:10448000DCE7511C9942C0F299819B1A924901EBD9
:10449000431122463846FFF709FC0546CEE74FF0A8
:1044A000E023D3F8F03D13F0010F00D000BE00234D
:1044B0001D46C3E7082B1AD0092B26D0062B40F047
:1044C000888021463846FFF7EBFC0546B6E72046D4
:1044D00000F070FB6188C9B23846FFF767FA784A86
:1044E000137843F00203137001231D46A6E7744BB3
:1044F0005B788DF8063001230DF10602214638461F
:1045000000F0F0FA01231D4698E76388DAB290467E
:104510006B4B5B78934231D0694B5B7863B9684BE6
:10452000414683F8018039B33846FFF7CDFB054695
:1045300080B1FFF72DFD21E000213846FFF796FA04
:104540003846FFF7C4FA5E4DAE783846FFF760FB99
:10455000AE70E4E74FF449725A495B48FEF716FE25
:104560004FF0E023D3F8F03D13F0010F00D000BE70
:10457000534B00225A7061E7FFF70BFD2146384686
:1045800000F09CFA01231D4658E76388012B02D0F6
:1045900000231D4652E74A4A137843F0080313707C
:1045A0002146384600F08AFA01231D4646E7638813
:1045B000012B02D000231D4640E7414A137823F027
:1045C000080313702146384600F078FA01231D468F
:1045D00034E74FF0E023D3F8F03D13F0010F00F083
:1045E000F08000BE00231D4628E7A388DAB20F2A18
:1045F00000F2EA80324A52FA83F31B79344A127885
:10460000934223D2334A116811EB431100F0DF804B
:1046100022463846FFF74AFB054600287FF40EAFD6
:10462000237813F0600F7FF409AF63780A3B012B06
:104630003FF604AF00F0B8FA63780A2B0FD021469A
:10464000384600F03BFA01231D46F7E6511C99421B
:10465000C0F2C0809B1A204901EB4311D8E7002328
:104660008DF8063001230DF106022146384600F090
:1046700039FA01231D46E1E6A288D1B202F07F0C8F
:10468000C2F3C01012F0700F28D10D4A02EB4C0299
:104690000244127D0E480078824230D20D480068F4
:1046A00000EB42121546002B36D02946002D3FF470
:1046B000C5AE22463846FFF7F9FA0546BEE600BF0A
:1046C0001414002054820010207E00104D3200107F
:1046D000DD1E002044120020A082001040F295321E
:1046E00041494248FEF752FD4FF0E023D3F8F03D38
:1046F00013F0010F00D000BE00231D469EE600F11E
:10470000010C944505DB121A394800EB421215469C
:10471000C9E700221546C6E76378012B11D0032BA9
:104720000FD093BB3846FFF72BFEADF806000223EF
:104730000DF106022146384600F0D4F901231D464A
:104740007CE6628822B9012B1BD03846FFF7DCFDDE
:10475000002D42D0224629463846FFF7A7FA00200E
:1047600000F022FA234B93F8353013F001031D4675
:104770007FF464AE2146384600F0A0F901231D46BF
:104780005CE63846FFF7DEFDE2E74FF0E023D3F8C2
:10479000F03D13F0010F00D000BE00231D464DE692
:1047A0004FF0E023D3F8F03D13F0010F18D000BE16
:1047B00000231D4642E600231D463FE600231D461A
:1047C0003CE600231D4639E600231D4636E600235D
:1047D0001D4633E600231D4630E601231D462DE627
:1047E00000231D462AE600BF54820010207E0010E0
:1047F000A08200101414002010B584B0FFF7DCFB79
:1048000000285AD104B010BD042B40F00081854B24
:104810001B7813F0010F50D0824B1878C0F3C00002
:10482000FFF7B8FB49E0072B00F08A80082B00F067
:10483000DD80062B40F0EB807B4B1B78002B6FD08C
:10484000794A1378013BDBB213701378ABBB754B1D
:104850001A7842F001021A7093F8342022F0010213
:1048600083F8342093F8342022F0040283F83420B3
:1048700093F8352022F0010283F8352093F8352093
:1048800022F0040283F8352002A99DF80400FFF706
:1048900085FD90B901469DF80400FFF733F98021AA
:1048A0009DF80400FFF72EF907E09DF80400FFF7DC
:1048B000F7F99DF808205B4B9A705C4B1C686369A4
:1048C000EFF3108272B6D3E8CF0F01210028FAD19E
:1048D000C3E8401F0028F6D1BFF35F8FA26101A992
:1048E000204601F0B2FB6169A3690022C1E88F2F65
:1048F00083F31088002885D09DF80530052B6CD0F7
:1049000091D8032B79D03FF67FAF012BCDD0022B6E
:104910007DD19DF80400FFF7C3F9FFF73AFBCCE720
:1049200040F2652242494348FEF730FC4FF0E02355
:10493000D3F8F03D13F0010F3FF464AF00BE61E720
:104940009DF8081001F07F00CC09364B03EB4003C3
:1049500003EBD11393F8342022F0010283F83420C2
:1049600093F8342022F0040283F83420A8B12D4BB0
:1049700003EB400323441B7D2F4A1278934214D249
:104980002E4A126812EB431317D09C69039B9DF8C3
:1049900009209DF80400A0478FE7039B9DF809209C
:1049A0009DF8040000F014F987E7501C984204DBDE
:1049B0009B1A234A02EB4313E7E74FF424721C4986
:1049C0001C48FEF7E3FB4FF0E023D3F8F03D13F073
:1049D000010F3FF417AF00BE14E7124B1B7813F022
:1049E000010F3FF46AAFFFF7D6FA66E7029B002B90
:1049F0003FF463AF039898475FE70A4BDB7813F007
:104A0000010F3FF45AAF0298FFF745FA55E74FF010
:104A1000E023D3F8F03D13F0010F3FF44EAF00BE9A
:104A20004BE700BF14140020DF1E00206C14002090
:104A300080820010207E0010DD1E00204412002025
:104A4000A082001008B591F90030002B05DB802111
:104A500000231A46FFF706FC08BD0021F8E7000016
:104A6000F8B50746134B9E89DD89741BA4B2402C10
:104A700028BF402493F90030002B08DB0021AE4210
:104A800013D00D4A23463846FFF7ECFBF8BDAE4283
:104A900009D0084B9968402C09D82246064802F0F4
:104AA000A9FB8021EBE78021E9E70022EAE700206B
:104AB000ECE700BFD41300209413002008B586460D
:104AC0000B46074A944608684968ACE80300002191
:104AD0009160D181918119467046FFF7B3FF08BDFF
:104AE000D413002038B505468C461446264A96460F
:104AF00008684968AEE8030094600021D181BCF8E1
:104B000006108B4228BF0B469381BCF8062032B3B7
:104B100003B134B12846FFF7A3FF044688B120460D
:104B200038BD722219491A48FEF730FB4FF0E023D6
:104B3000D3F8F03D13F0010F00D000BE00231C4657
:104B4000EDE7742211491248FEF720FB4FF0E023F5
:104B5000D3F8F03D13F0010FE1D000BEDFE761466E
:104B60002846FFF76FFF04460028D8D17622074970
:104B70000748FEF70BFB4FF0E023D3F8F03D13F0AE
:104B8000010FCCD000BECAE7D4130020F882001079
:104B9000207E0010034B00221A605A609A60DA608F
:104BA0001A617047D4130020014B1861704700BF91
:104BB000D41300200146054B1A460068496803C219
:104BC00000229A60DA819A81704700BFD4130020D6
:104BD00038B504461A461D463E4B1B78DB09B3EB3D
:104BE000D11F1ED082B19D223B493C48FEF7CEFA30
:104BF0004FF0E023D3F8F03D13F0010F00D000BEDA
:104C000000231C46204638BD3249FEF73DFF314B9C
:104C10001B691BB12F4A03212046984701231C46DC
:104C2000F0E72C4B93F90030002B06DB294B9868FA
:104C300000284CD02A4902F0DDFA264AD38913FA1B
:104C400085F39BB2D381916829449160D2889342C5
:104C500001D03F2D27D81F4B1B6923B11D4A0221CC
:104C600020469847A0B11B492046FFF7EBFE0446BB
:104C70000028C7D1C52218491848FEF787FA4FF017
:104C8000E023D3F8F03D13F0010FBBD000BEB9E72D
:104C900001462046FEF736FF80212046FEF732FF10
:104CA00001231C46AEE72046FFF7DAFE0446002843
:104CB000A8D1CD2208490948FEF768FA4FF0E02351
:104CC000D3F8F03D13F0010F9CD000BE9AE70446E4
:104CD00098E700BFD4130020E0820010207E00106F
:104CE0009413002070B50446FFF756F918B9002355
:104CF0001E46304670BDFFF757F906460028F6D12C
:104D00001C4BC82202FB0433DB78002BEFD0C823F6
:104D100004FB03F31033174A13441D46184601F0F1
:104D20007EF93F28E5D9134BC82202FB0433D9781A
:104D30000020FFF76FFA08B90646DAE7284601F0C7
:104D40006EF93F280DD90B49C82303FB04114023FA
:104D5000094A02EBC412C9780020FFF783FA06461D
:104D6000C7E7044BC82202FB0433D9780020FFF7C1
:104D700065FABEE7CC1200204812002010B50446A8
:104D8000FFF70AF900B910BDFFF70EF948B9074B54
:104D9000C82202FB04331B7913F0010F03D001205A
:104DA000F1E70020EFE70020EDE700BFCC12002084
:104DB00008B5C82303FB00F01030024B184401F083
:104DC000FDF808BDCC12002038B50446C82300FB0E
:104DD00003F31033084818444FF6FE739A4208D87C
:104DE00092B201F051F905462046FFF77BFF2846B5
:104DF00038BD4FF6FF72F4E7CC12002070B50446C0
:104E0000FFF7CAF808B9002070BDFFF7CDF80028F9
:104E1000F9D1C82304FB03F32033224A134404339B
:104E20001E46184601F0CAF80028EDD01D4BC822D6
:104E300002FB043399780020FFF7ECF90028E3D057
:104E4000E3014033184A13441D46402219463046B8
:104E500001F01AF90646D8B11249C82303FB041120
:104E600003462A4689780020FFF7FCF908B130464E
:104E7000CAE7D5220D490E48FEF788F94FF0E02326
:104E8000D3F8F03D13F0010F00D000BE0020BBE7C7
:104E9000044BC82202FB04339978FFF7CFF90020B6
:104EA000B2E700BFCC120020481200202883001077
:104EB000207E001070B50646C82400FB04F42034A0
:104EC0000C4B1C4404344FF6FE739A420BD892B23A
:104ED000204601F010F90546204601F06FF83F2802
:104EE00004D8284670BD4FF6FF72F1E73046FFF751
:104EF00085FFF6E7CC12002008B5C82303FB00F0BD
:104F00002030034B1844043001F089F808BD00BF7D
:104F1000CC1200202DE9F04383B0C82200212148A3
:104F200002F00CF90025204B1D7015B103B0BDE84F
:104F3000F0831C4FC82405FB04F43E19FF23737152
:104F40004FF4E133B360357375730823B37304F121
:104F5000380104F1100000950123402239443844FF
:104F600000F0FBFF04F1780104F120003844012334
:104F7000009340223944043000F0EFFF04F1B809F7
:104F8000B9444846FBF7DEFDC0343C442046FBF7FD
:104F9000D9FDF561C6F82090346375630135EDB233
:104FA000C3E700BFCC120020C812002000230BB1C1
:104FB000012070479C460C4AC82101FB0322116A5C
:104FC000106B29B1084AC82101FB0322D361136287
:104FD00030B1054AC82101FB0C2200211163516345
:104FE0000133DBB2E3E700BFCC12002038B5002468
:104FF00004B138BD2546C82304FB03F317495818EC
:10500000CC500471164B1B7813F0010F12D0144BC7
:105010001B7813F0020F16D0C823284603FB00F0BC
:1050200020300E4B18440121043001F084F8013483
:10503000E4B2DDE7C82304FB03F310330846184449
:1050400001F05EF8E3E7C82005FB00F02030034BD9
:105050001844043001F054F8DEE700BFCC12002001
:10506000C81200202DE9F04182B04B79022B40F0AC
:10507000818007468B79022B40F0818000231E46F9
:105080003EB19EB98B7888F800300B78CC18092592
:1050900020E0C8203B4B00FB063398469B78002B52
:1050A000EFD033460133DBB21E46E9E740F241124E
:1050B00035493648FEF76AF84FF0E023D3F8F03D63
:1050C00013F0010F00D000BE002554E023781D44EA
:1050D000ADB21C446378242B01D19542F6D9052B3F
:1050E00009D06378042B02D163790A2B20D0304693
:1050F000FFF7F8FD3FE021463846FEF7FBFF38B1E9
:10510000A37888F8013023781D44ADB21C44E8E749
:1051100040F253121C491D48FEF738F84FF0E023C7
:10512000D3F8F03D13F0010F00D000BE002522E0BF
:1051300021780D44ADB24246931C0193D31C0093D9
:1051400002231A4621443846FFF714F810B10E35F1
:10515000ADB2CCE74FF4B1720B490C48FEF716F82C
:105160004FF0E023D3F8F03D13F0010F00D000BE64
:10517000002500E00025284602B0BDE8F0810025AA
:10518000F9E700BFCC1200201C830010207E001025
:10519000137803F06003202B7CD170B59446002473
:1051A00074B1002C78D19CF80130222B42D017D852
:1051B000202B1FD0212B11D1012933D001206CE0ED
:1051C000C82304FB03F3384A03EB020ED25CBCF89D
:1051D00004309A42E5D00134E4B2E1E720465CE0D5
:1051E000232B05D1012947D003294AD0012054E0BF
:1051F000002052E0012903D0032909D001204CE00E
:1052000007230EF108026146FFF76CFC012044E021
:10521000264B002B42D00EF108012046FEF734F851
:1052200001203AE007230EF108026146FFF75AFC1D
:10523000012032E0012903D0032906D001202CE00F
:105240006146FFF73BFC012027E0BCF8023003F089
:105250000105C3F340068EF8043085F001010EF11C
:10526000240000F068FF124BD3B132462946204695
:10527000AFF30080012010E06146FFF71FFC012022
:105280000BE00C4B73B1BCF802102046AFF300806A
:10529000012002E000207047002070BD0120FCE7E3
:1052A0000120FAE70120F8E7CC1200208932001033
:1052B00000000000000000002DE9F84F82460D4676
:1052C000984600245CB1BCB9A146F378AB4223D028
:1052D000B378AB4254D001242046BDE8F88FC823F0
:1052E0003C4E03FB0466F378AB42ECD0B378AB42A0
:1052F000E9D00134E4B2E5E74FF4E67236493748C5
:10530000FDF744FF4FF0E023D3F8F03D13F0010F19
:1053100000D000BE0024DFE706F110039B461FFA11
:1053200088F22F4901EBC411184600F0E4FE2D4B22
:10533000C3B17379FF2B15D0002700E00137474533
:1053400010D27279264B03EBC913DB5D9A42F5D17B
:10535000584600F047FE0028F0D171792046AFF39F
:105360000080EBE7204B1BB1584600F03BFE18B124
:105370002046FFF7B7FCABE72046AFF30080F7E726
:105380001A4B13B12046AFF300802046FFF736FDDD
:1053900008B10124A0E706F1240000F00FFEA8B92F
:1053A0004346ABB118F03F0F01D0012494E7B17828
:1053B0005046FEF72FFF044608B901248CE700236E
:1053C0001A46B1785046FEF74DFF85E7012483E782
:1053D000012481E7CC1200200C830010207E0010F5
:1053E0004812002000000000000000000000000043
:1053F00090B90A4B4FF4137101FB003393F8293134
:1054000033B9064B01FB00335B791BB101207047B8
:10541000012070471846704700207047B0150020E3
:1054200008B10020704708B54FF41372034902FB1E
:105430000011043100F036FB08BD00BFB01500209C
:105440002DE9F04784B04FF4137200211E4801F09B
:1054500075FE002414B104B0BDE8F0874FF4137555
:1054600004FB05F505F5A473174F3B440433E6012F
:10547000DFF858A00AEBC41205F594704FF040090C
:10548000CDF80C9002924FF48078CDF80480009310
:10549000234622462146384400F08EFA05F12003C7
:1054A0003B4408334E445644E819CDF80C9002961C
:1054B000CDF804800093234601222146043000F0F9
:1054C0007BFA0134E4B2C5E7B015002030150020A6
:1054D00070B500240CB1012070BD4FF4137504FBAE
:1054E00005F505F59470054E304400F08EFAA819C4
:1054F000043000F08AFA0134E4B2EBE7B015002082
:105500002DE9F04100250DB1BDE8F0814FF4137491
:1055100005FB04F40A4E04EB0608355504F59870B3
:10552000304400F0EDFD04F108003044043000F098
:10553000E7FD88F8295188F805500135EDB2E2E71A
:10554000B01500204B79FF2B40F095802DE9F041FC
:1055500082B080460F460C780C44A51800261EB178
:10556000002002B0BDE8F0813046FFF741FF10B1E6
:105570000136F6B2F3E74FF4137306FB03F33F4A29
:1055800099180191B978D1542BE0AC4270D22146E0
:105590004046FEF7AFFD78B30136F6B2A378DB09DB
:1055A00039D1019A02F5987000F0AAFDA37801990B
:1055B00081F82931A388C3F30A03B3F5007F14BF30
:1055C0000023012391F8282163F3410281F8282167
:1055D00001F59471404600F0AFFA002839D02378E5
:1055E0001C443B79B34243D96378052BCDD0AC4200
:1055F000CBD223781C44F7E7E02221492148FDF76C
:10560000C5FD4FF0E023D3F8F03D13F0010F00D0BB
:1056100000BE0020A5E7019A02F10C0000F070FD29
:10562000A37801994B71A388C3F30A03B3F5007FF4
:1056300014BF002301230A7963F341020A710F4862
:10564000081A8010104B03FB00F0C0B2FFF7E8FE11
:10565000C5E7E8220A490B48FDF798FD4FF0E02323
:10566000D3F8F03D13F0010F00D000BE002078E722
:10567000E11B88B275E70020704700BFB01500201D
:1056800040830010207E00109B1DB5082DE9F041DD
:1056900006461F4600245CB1002C48D1A04695F870
:1056A00029318B4213D06B798B422BD001203FE004
:1056B0004FF413731F4D03FB045595F829318B42AA
:1056C000EAD06B798B42E7D00134E4B2E3E7B5F876
:1056D00034317BB9184B33B1BAB2184901EBC81158
:1056E0002046AFF3008005F59471304600F024FAAF
:1056F00001201DE0BAB2D5F82C1105F5987000F024
:10570000FAFCE7E70E4B1BB1B9B22046AFF30080BD
:1057100004352946304600F0C5F908B1012007E0FC
:105720003A462946304600F073F9012000E0002097
:10573000BDE8F081B0150020000000003015002009
:105740000000000010B582B059B10A46012825D8E2
:105750000B781BB324490B54012B31D001231C4679
:105760002BE001238DF8043008468DF8051001A9BF
:10577000FEF72AFC044618B11B4B01221A701CE0EC
:1057800047221A491A48FDF701FD4FF0E023D3F8EC
:10579000F03D13F0010F10D000BE0EE05A22134965
:1057A0001348FDF7F3FC4FF0E023D3F8F03D13F07E
:1057B000010F00D000BE00231C46204602B010BDE1
:1057C0001146FEF701FC04460028F6D15F22074986
:1057D0000748FDF7DBFC4FF0E023D3F8F03D13F072
:1057E000010FEAD000BEE8E708140020C0830010D3
:1057F000207E001070B50446037813F0010022D11A
:105800008C460D462378C3F38002164613F0040F2E
:105810001AD14FF0FF31604601F0E2FD237813F01A
:10582000010309D1227812F0040F0AD1237843F042
:105830000403237001231E46284601F0DDFD304697
:1058400002E01E46F8E7002070BD70B5044606462B
:105850000A460D464FF0FF31104601F0C1FD237896
:10586000C3F38002144613F0040F04D1284601F05C
:10587000C3FD204670BD337813F0010F04D1337897
:1058800023F004033370F1E700231C46EEE7000029
:1058900008B58388C3F30A02C37803F00303022B1D
:1058A0001DD0032B44D0012B5BD1022905D040F23F
:1058B000FF33934204D3012054E04FF48063F8E7B0
:1058C000D12229492948FDF761FC4FF0E023D3F8A4
:1058D000F03D13F0010F00D000BE002042E002298D
:1058E00003D0402A15D801203CE0B2F5007F01D159
:1058F000012037E0D8221C491C48FDF747FC4FF037
:10590000E023D3F8F03D13F0010F00D000BE0020DB
:1059100028E0DB2214491548FDF738FC4FF0E0235E
:10592000D3F8F03D13F0010F00D000BE002019E0C5
:10593000022904D04023934204D3012012E04FF403
:105940008063F8E7E12208490848FDF71FFC4FF0A3
:10595000E023D3F8F03D13F0010F00D000BE00208B
:1059600000E0002008BD00BFAC830010207E0010C6
:105970000A4403E000BD91F800C0614491421AD28C
:1059800091F801C0BCF1050FF5D100B591F802C046
:105990000CF07F0E00EB4E0E4FEADC1C0EF80C30C4
:1059A00091F800C061449142E4D291F801C0BCF189
:1059B000050FF5D1EAE7704770B582B00446164688
:1059C000BDF81C5090F800C061F3000C00F808CB43
:1059D000009301232A46069900F0BFFA069B03B103
:1059E0003DB9089B6360BDF824306380012002B09C
:1059F00070BD04F11C052846FBF7A4F833460EB130
:105A00002B4600256361A561EBE70120704700008C
:105A1000F8B507460C4615460B7813F0020F11D067
:105A20004FF400731E4604F1080000F0C7FA70BB83
:105A30007DB3731E2B422ED1237813F0010F04D0B7
:105A4000002025E040231E46EDE761783846FEF74A
:105A5000E1FB0028F4D0237813F0010F0FD04FF4AE
:105A6000B5720E490E48FDF791FB4FF0E023D3F8D5
:105A7000F03D13F0010F00D000BE002008E000232D
:105A80001A4661783846FEF7EDFB08B9E7E70020D3
:105A9000F8BD2846FCE70020FAE700BF8883001025
:105AA000207E001070B505460C4601F108031E4625
:105AB000184600F083FA20B1237813F0010F01D0CB
:105AC000002070BD61782846FEF7A4FB0028F7D0BF
:105AD00062886168304600F0D7FA0646E8B123785C
:105AE00013F0010F0FD04FF4BC7211491148FDF7AC
:105AF0004DFB4FF0E023D3F8F03D13F0010F00D041
:105B000000BE0020DDE70346626861782846FEF7A4
:105B1000A9FB0028E7D03046D3E7237813F0010F24
:105B200001D00020CDE761782846FEF787FBF8E733
:105B30006C830010207E0010F8B505460C468B895A
:105B40005BBB0B7813F0010F01D00020F8BD497842
:105B5000FEF760FB0028F8D06388227812F0010F6E
:105B60000FD04FF4D9723A493A48FDF70FFB4FF086
:105B7000E023D3F8F03D13F0010F00D000BE002069
:105B8000E4E761783BB162682846FEF76BFB0028CA
:105B9000E7D06088DAE71A46F6E70B7813F0020FD1
:105BA00010D04FF400731E4604F108031F46184638
:105BB00000F035FA864248D8237813F0010F04D05C
:105BC0000020C3E740231E46EEE761782846FEF733
:105BD00021FB0028F4D0384600F021FA864229D86B
:105BE00073429AB2618802EA00038B4228BF0B46D7
:105BF0001E46237813F0010F0FD040F2C71214494C
:105C00001448FDF7C3FA4FF0E023D3F8F03D13F04A
:105C1000010F00D000BE002098E7617846B16268AD
:105C200033462846FEF71EFB0028E6D030468DE7B7
:105C30003246F5E7237813F0010F01D0002085E705
:105C400061782846FEF7FAFAF8E700207EE700BF01
:105C500050830010207E001003460A4490B2814217
:105C600002D8B0EB430F03DB5B009BB2C01A80B2DB
:105C7000704710B50C46B0F804C09A420DD3A2EBA1
:105C8000030E1FFA8EF121B38C4515D294450DD821
:105C9000A2EB0C0293B243810EE0A2EB030E4FEA9B
:105CA0004C0111FA8EFE1FFA8EF1ECE7624493B2BA
:105CB000F1E7A3EB0C039BB29C45FAD90168C288BB
:105CC000C2F30E0202FB0311204601F093FA0120F9
:105CD00010BD0846FCE72DE9F84304460F469DF841
:105CE0002050B0F804C0ACEB030080B2A3EB0C0C66
:105CF00094441FFA8CFCE188C1F30E0E76461EFB1D
:105D000000F189B288461EFB0CFE1FFA8EF189460F
:105D1000216806FB031135B9904206D306FB02F257
:105D2000384601F067FABDE8F8834246384601F08C
:105D300061FA4A4621683846404401F05BFAF2E7CE
:105D400030B583B015469E46BDF81830B0F804C093
:105D50009E4511D3AEEB0304A4B224B3A44507D2ED
:105D6000F44511D8AEEB0C0E1FFA8EF34381644656
:105D7000AC4210D32C460EE0AEEB03044FEA4C02CB
:105D800012FA84F4A4B2E8E7E6441FFA8EF3EDE7D2
:105D9000A3EB0C039BB29C45FAD99DF81C20009202
:105DA0002246FFF798FF204603B030BDF0B583B020
:105DB00004460D4616461F46006918B14FF0FF31E4
:105DC00001F00EFB2389628992B2019700929BB287
:105DD000324629462046FFF7B3FF02460546618951
:105DE00089B2A088FFF738FF6081206908B101F00F
:105DF00003FB284603B0F0BD2DE9F04104460F46F1
:105E00009DF818E0B0F804C0ACEB030189B2A3EB35
:105E10000C0C94441FFA8CFCC588C5F30E00054693
:105E200010FB01F610FB0CF080B28046206805FBE9
:105E30000300BEF1000F07D1B6B2914206D305FBB5
:105E400002F2394601F0D6F9BDE8F0813246394612
:105E500001F0D0F9424639463144206801F0CAF9D0
:105E6000F2E72DE9F04383B01646002A73D00446CA
:105E700089469846C06818B14FF0FF3101F0B0FA7A
:105E800023899AB21746B4F80AC01FFA8CF1E37955
:105E9000DB091DD1A5888A4212D3A2EB010C1FFA9F
:105EA0008CFC654555D9A5EB0C05ADB23346AE4229
:105EB00028BF2B461D46002D43D0A2883B4631E02B
:105EC000A2EB010C6B0013FA8CFC1FFA8CFCE8E7C8
:105ED000A588B5420AD84246F2B9721BE388C3F3DB
:105EE0000E0303FB029399460F46E4E78A420DD363
:105EF000531A9BB23344B3EB450F0FDBAA1B92B28C
:105F00002846FFF7A9FE07463546D4E7531A6A002C
:105F100012FA83F39BB2EDE70F46CCE73546CAE7AA
:105F20009B1A9BB29A42FBD9CDF800802A4649467B
:105F30002046FFF761FF2A463946A088FFF78CFE0E
:105F40002081E06808B101F057FA284603B0BDE8A7
:105F5000F0830025F5E71546F7E7F8B51F46B2F5DB
:105F6000004F27D804460D461646C06818B14FF0BA
:105F7000FF3101F035FA206918B14FF0FF3101F01F
:105F80002FFA2560A680E38867F30E03E380E379A8
:105F90009DF8182062F3C713E37100236381238106
:105FA000E06808B101F028FA206928B101F024FA6C
:105FB0000120F8BD0020FCE70120FAE702468088B6
:105FC00013899BB2528992B2934205D39B1A9BB21A
:105FD000984228BF184670479B1A420012FA83F372
:105FE0009BB2F5E7028992B243899BB29A4214BFF1
:105FF000002001207047818803899BB2428992B2B8
:10600000934206D39B1A98B281428CBF0020012094
:1060100070479B1A4A0012FA83F398B2F4E7828819
:1060200003899BB2418989B28B4206D35B1A9BB22A
:106030009A4208D9D01A80B270475B1A510011FAFF
:1060400083F39BB2F4E70020704738B504460D4651
:10605000006918B14FF0FF3101F0C2F9228963895C
:106060009BB292B229462046FFF703FE0246054640
:10607000618989B2A088FFF7EFFD6081206908B1CE
:1060800001F0BAF9284638BD08B50023FFF78EFEA7
:1060900008BDF8B504460F46C06818B14FF0FF318F
:1060A00001F09EF923899BB21D462046FFF7A3FF0E
:1060B00018B1E379DB091E4617D0A2882B4601E010
:1060C0009B1A9BB29A42FBD92068E288C2F30E0267
:1060D000394602FB030001F08DF801222946A08811
:1060E000FFF7BAFD208101231E46E06808B101F0E8
:1060F00083F93046F8BD08B50023FFF7B2FE08BDAE
:1061000010B50446C06818B14FF0FF3101F068F9CE
:10611000206918B14FF0FF3101F062F9002363816B
:106120002381E06808B101F067F9206908B101F046
:1061300063F9012010BD38B504460D46C06818B19A
:106140004FF0FF3101F04CF9206918B14FF0FF31E9
:1061500001F046F9E37965F3C713E371E06808B12C
:1061600001F04AF9206908B101F046F9012038BD73
:10617000074B98420AD0132301229A40054B1A601C
:10618000054B9B6832EA0303FAD170471223F3E709
:1061900000000840003002400000024070B5054693
:1061A0000C460620FBF7E2F9AE465EF8046F06F0F7
:1061B00002060EF5405202231360FE2B09D81A0284
:1061C000A2FB042190424FF000028A4104D3023323
:1061D000F3E74FF4807101E04FF48071012909D990
:1061E00001F1FF3C03FB0CF2B0FBF2F2A24201D83A
:1061F0006146F3E72B614C1E2A6882EA042202F40E
:106200007F4205F580552A600EF5005ECEF80060ED
:1062100001FB03F3B0FBF3F070BD000038B504469A
:106220000D46174B984229D0132201239340154A5B
:1062300013602046FFF79CFF29462046FFF7AEFF7C
:10624000234653F8041F01F0020103F540524FF0BA
:10625000020CC2F800C0226882F0070202F0CF02EE
:1062600004F5805ECEF8002003F50053196004F5B4
:10627000005403226262C3F800C038BD1222D4E782
:10628000000008400020024000B583B003681B7C7A
:10629000D0F834C003FB01F1C90089B26144009118
:1062A000002100F0CDFE03B000BD2DE9F04106460F
:1062B00090F8387090F83950036893F811800024F2
:1062C0002A4621463046FFF7DFFF0134E4B20135AC
:1062D000EDB2A74201D9A845F2D8BDE8F08108B5D2
:1062E00003681B7C90F8382003FB02F2D2000021E7
:1062F000406B00F023FF08BD10B5044680F839104C
:10630000036B1B689847236B5B682046984710BD5A
:1063100010B5044690F8933023B900212046FFF7CA
:10632000EBFF10BDFFF7DBFFF7E738B50446FFF7DB
:10633000BCFF94F8393094F838501D44EDB223680E
:106340005B7CAB4208D994F8933053B92946204678
:10635000FFF7D2FF012038BD204600F097FE002055
:10636000F9E72046FFF7BBFFF0E708B5FFF79DFF11
:1063700008BD10B50446FFF7CBFF2046FFF7D5FF59
:106380000028FAD101462046FFF7B6FF10BD0000F5
:1063900030B585B005460C4600931346084A0949B6
:1063A00000F096FE0DF10F0000F0A2FE01460094F1
:1063B000054B9DF80F20284600F0AAFC05B030BD23
:1063C0002F6E0010616F0010496B0010405C704729
:1063D0004218435C507800EB032080B270470020E5
:1063E000704738B504460D4600212846FFF7EEFFFA
:1063F000207001212846FFF7E9FF6070022128463E
:10640000FFF7E4FFA07003212846FFF7DFFFE070ED
:1064100004212846FFF7DAFF207105212846FFF7FF
:10642000D5FF607106212846FFF7D0FFA071072134
:106430002846FFF7CBFFE07108212846FFF7C6FF8B
:10644000207209212846FFF7C1FF60720A21284601
:10645000FFF7BCFFA0720B212846FFF7B7FFE072E1
:106460000C212846FFF7B2FF20730D212846FFF7C5
:10647000ADFF60730E212846FFF7A8FFA0730F2120
:106480002846FFF7A3FFE07310212846FFF79EFF81
:10649000207411212846FFF79BFF608213212846B4
:1064A000FFF796FFA08215212846FFF791FFE082B3
:1064B00038BD10B5024690F80CE00468207840FA28
:1064C0000EF05FFA80FC0EEB0103DBB2072B11D953
:1064D000CEF1080E5FFA8EFE04F1010CC2F800C086
:1064E00094F801C00CFA0EFC4CEA000C5FFA8CFC2C
:1064F000083BDBB24FF0FF30884013732CEA0000FA
:1065000010BD38B5044600F160050166002380F82F
:106510006C3090F878102846FFF7CBFF84F86A00BB
:1065200094F879102846FFF7C4FF84F86B0094F8BC
:10653000923084F86E30B3FA83F35B0984F86F30DD
:1065400038BD10B50C46FFF7B4FF611EC9B2012378
:106550008B40C01A40B210BD012B05D0022B06D0D3
:1065600043B9104480B27047084480B27047801A23
:1065700080B27047401A80B27047012B05D0022BC1
:1065800006D043B9084480B27047801A80B2704781
:10659000401A80B27047104480B270472DE9F04F26
:1065A00089B005468A46079290F968305FFA83FB06
:1065B00090F96920D3B2049319E0CDF814A01FE03C
:1065C00095F86E3085F892300097059B069928461D
:1065D00000F028FAB2453CD3ABEB040454445FFA14
:1065E00084FA049B0133DBB204934FF0000B95F95E
:1065F0006A40E4B2A4EB0B06F6B2B245DDD30596D1
:10660000B5F866904FFA8BF19DF9108095F870708F
:106610003B4642460391B5F86400FFF7AEFF069093
:106620003B46424603994846FFF796FF0246079BC2
:10663000002BC5D195F86D30002BCBD195F86F307C
:1066400085F892300097059B0699284600F0EAF9F4
:10665000C0E70AEB0B0385F8683085F8698009B05C
:10666000BDE8F08F2DE9F04F85B0044600F16005DC
:10667000FFF747FF94F96B6094F87A102846FFF70C
:1066800060FF814694F87B102846FFF75AFF80464A
:1066900094F87C102846FFF754FF834694F96A70FB
:1066A000002F78DD06EB0803DBB25B425BB21A46D3
:1066B00094F87080434692464946B4F86400FFF768
:1066C0005CFF0390A4F86400434652464946B4F880
:1066D0006600FFF741FF0246A4F86600B8F1020F1A
:1066E0005DD013D8B8F1000F20D0B8F1010F0BD155
:1066F000039B991B89B2013101339BB210FA87F0D9
:1067000080B289B2039117E0039B15E0B8F1030F43
:106710000AD1039B33449BB2B9B2411A89B2013109
:10672000013080B28AB207E0039B05E0039B13FAB5
:1067300087F39BB2304480B200900399204600F06A
:10674000EDF940B3002384F8683084F8693094F898
:1067500076102846FFF7ADFE804694F8771028465D
:10676000FFF7A7FE0746002241462046FFF716FF27
:10677000012239462046FFF711FF01212846FFF785
:1067800098FE0028EFD194F96930B342DFDB94F82A
:106790006E3084F89230584605B0BDE8F08FB9B23B
:1067A000039B591A89B2013101339BB2871BBFB2D7
:1067B0000137013080B2BAB289B20391BCE770B53B
:1067C0000E46846D1734FF2913D8602903D9B0F819
:1067D00088301C4406E0402904D9B0F886301C44B7
:1067E00000E01C44637803B32278B242F9D1A01CC4
:1067F0001CE0B0F88A301C44254600212846FFF7EB
:10680000E7FD044402212846FFF7E2FD04358642F5
:10681000F3D801E0A3781C442278637853EA02237A
:1068200005D09E42F6D1E01C00E0184670BD002065
:10683000FCE710B50446A0F86410A0F866201946DD
:10684000FFF7BDFF20B101462046FFF70BFF80B2E6
:1068500010BDF8B504460D4616461F4690F8703038
:10686000022B1FD008D883B1012B14D1C36D9847D8
:10687000281A83B21D460EE0032B0CD1C36D984736
:106880002B4603449BB21D4605E0C36D9847334633
:1068900003449BB21E463B46324629462046FFF73C
:1068A000C8FFF8BDC36D9847301A83B21E46F2E7A1
:1068B0002DE9F04104460F4616461D4600F057FAF2
:1068C0004FF0000809E0032B04D1361AB6B201E0FC
:1068D0000744BFB240441FFA80F863682978204615
:1068E00098474FF6FF72904219D001354FF6FE726D
:1068F0009042F2D00346324639462046FFF7A9FFC0
:1069000094F87030022B07D0DDD8002BE0D0012B9B
:10691000E0D10644B6B2DDE73F1ABFB2DAE740463F
:10692000BDE8F08108B5DFF80CC0C0F804C0FFF77F
:10693000BFFF08BD596D0010836D63B390F98120CE
:1069400080F88E2090F9823080F88F3090F88D108A
:1069500009B3012912D000B590F97EC090F98010DA
:106960000CEB010E724504DACAB252FA8CFC80F8C4
:106970008EC08B4201DD80F88F1000BD90F983102E
:106980008A4201DA80F88E1090F98420934202DD69
:1069900080F88F2070477047014BC365704700BF78
:1069A000DF630010836D8B4209D010B5044681650A
:1069B0007430FFF716FD2046FFF7BEFF10BD70478D
:1069C00000B5B0F800E0B1F800C0F4441FFA8CFC48
:1069D000E64505D99E4512D203F1FF3C1FFA8CFC17
:1069E0009E450ED294450ED9964500D372469C45DD
:1069F00000D8634602809B1A0B80012000BD96469A
:106A0000EEE70020FAE70020F8E710B582B0C48F67
:106A1000121BC46A9DF810C0CDF800C092B2A04706
:106A200002B010BD30B585B004469DF82000ADF829
:106A30000E10ADF80C20ADF80A3094F88C3063B32A
:106A4000BDF80A304BB3012B03D9022827D0032805
:106A50002ED010F001031D4634D1B4F84C20BDF8FF
:106A60000C309A4219D8B4F84E20934215D2B4F89B
:106A70004A30B4F848200DF10A010DF10E00FFF77D
:106A80009FFF50B12046236B9C680095BDF80A30EB
:106A9000BDF80C20BDF80E10A04705B030BD8AB27D
:106AA000D31A9BB2ADF80E300133ADF80E30D0E7FB
:106AB000BDF80C20D31A9BB2ADF80C300133ADF801
:106AC0000C30C6E7B4F84820BDF80E309A42E4D83E
:106AD000B4F84A209342E0D2B4F84E30B4F84C20D7
:106AE0000DF10A0103A8FFF76BFF0028CAD1D4E714
:106AF0008A4205D2834209D89A4209D901207047B7
:106B0000834207D99A4207D9012070470120704774
:106B100000207047002070470020704770B5044681
:106B20000E461D46BDF81030B0F84E10B0F84C00BF
:106B3000FFF7DEFF38B12B463246B4F84A10B4F8FE
:106B40004800FFF7D5FF70BD70B504469DF81050A2
:106B500002F0070E4FF0010C0CFA0EFC5FFA8CFCF1
:106B600090F89260012E1BD90020012E1AD022F03D
:106B7000070292B22668367C16FB02F292B20A44F1
:106B8000616B1144DDB90A780243D2B20A7082EA1D
:106B90000C0201F8012B013B9BB2002BF3D170BD1D
:106BA0006046E2E74FF0000CE1E701201BE0400007
:106BB000C0B24FEA4C0C5FFA8CFC002BEFD00A7885
:106BC0000243D2B20A7082EA0C020A700EF101028C
:106BD000013B9BB212F0070EE9D1628F114494F889
:106BE0009220012AE1D9012AE7D04FF0010CE4E715
:106BF00010B5016890F83830DA0082870A7CD2003C
:106C0000428790F839E04FEACE02C28703EB0E04C8
:106C100091F811C0644503DDACEB0E0C1FFA8CF348
:106C2000DB009BB2A0F84020A0F842201A44A0F854
:106C300042208B8AA0F84430CB8AA0F8463010BDA1
:106C400008B5FFF7D5FF08BD10B582B00446B0F80F
:106C500056300093B0F85230B0F85420B0F85010CD
:106C6000FFF75CFF18B984F88C0002B010BD012357
:106C700084F88C30B4F84820B4F850309A4201D2ED
:106C8000A4F84830B4F84A20B4F852309A4201D9F6
:106C9000A4F84A30B4F84C20B4F854309A4201D2E7
:106CA000A4F84C30B4F84E20B4F856309A42DCD9EF
:106CB000A4F84E30D9E708B50022A0F84820B0F873
:106CC0004420A0F84A20B0F84020A0F84C20B0F8AA
:106CD0004220A0F84E20FFF7B7FF08BD00B583B0F3
:106CE0009DF810C0CDF800C0FFF78FFE03B000BDC7
:106CF00008B50022A0F85020A0F854204FF6FF72EB
:106D0000A0F85220A0F85620036B5B68984708BD96
:106D100038B504469C46049B00258565C0F82CC008
:106D2000416380F8382080F8395080F86D5080F841
:106D3000915080F88D50012280F8922080F89320A5
:106D400003631B6898472046FFF7D2FF2046FFF7F2
:106D500023FE84F8705038BD084611B10A2903D0CB
:106D600070474FF6FF7070474FF6FF707047002373
:106D700080F82630704710B50A46C46800231521F4
:106D8000A04710BD10B50A46C46800231621A047CD
:106D900010BD10B51346C4680A461721A04710BDA0
:106DA00010B5C46800231A461821A04710BD10B5BD
:106DB000C46800231A461921A04710BD70B582B0DF
:106DC00006460D4609E015292FD322788DF80720B5
:106DD000F46800233046A04702352C4614F8011B06
:106DE000192910D8182919D21629ECD917291CD11C
:106DF0006B788DF807300DF1070201213046FFF75F
:106E0000C8FF0235E9E7FE290FD122788DF8072067
:106E10002921304600F041F90235DEE7F56800230C
:106E20001A463046A8472546D7E702B070BDF8B5E8
:106E30000546164616291BD00C461F460ED81429A7
:106E400022D0152908D1002100F058F931462846F2
:106E500000F062F901201EE000201CE0172910D08C
:106E60001AD3A1F11803DBB2012B0DD9002012E0D7
:106E7000002100F043F93146284600F04DF9012089
:106E800009E0012100F03AF928462B691D463B46EE
:106E900032462146A847F8BD0020FCE7F0B583B094
:106EA000054614460E2948D01F460F2904D00B2949
:106EB00038D0002003B0F0BDFFF772FF7B79DB0014
:106EC000DBB295F822101944CEB2C1F3031141F0A0
:106ED00010012846FFF74FFF019606F00F012846E4
:106EE000FFF749FFB97941F0B0012846FFF743FFAA
:106EF0003E79F600F6B23F68019AB318842B03D9A5
:106F00006FF07B039B1ADEB23A4631462846FFF704
:106F100040FF631E13F0FF04F6D12846FFF747FF3A
:106F20000120C7E722B90C49FFF748FF0120C1E75C
:106F30000A49FFF743FF0120BCE7FFF731FF81213A
:106F40002846FFF718FFA1082846FFF71BFF284631
:106F5000FFF72DFF0120ADE710A3001008A30010DC
:106F600070B504460D461646FFF798FF48BB0A2D3C
:106F700009D00D2D10D0092D24D11349204600F041
:106F80002BF801201EE0204600F02BF80F49204688
:106F9000FFF714FF012015E04EB90D492046FFF719
:106FA0000DFF23689B7C84F8223001200AE0094908
:106FB0002046FFF703FF2368DB7C84F822300120A2
:106FC00000E0012070BD00BFE0A20010BCA20010D4
:106FD00000A30010F8A2001001608B7C80F8223022
:106FE000704738B5044600231A4628214569A8474A
:106FF00000231A4614212046E568A84701224B21A8
:10700000204600F04AF823681A792921204600F02A
:1070100044F800224B21204600F03FF823681A79FB
:107020002921204600F039F801224B21204600F0AA
:1070300034F823685A792921204600F02EF838BD0B
:1070400010B582B08DF805108DF806208DF804304B
:10705000049B009384686B4601220F21A04702B075
:1070600010BD10B5846800231A460921A04710BD41
:1070700010B5846800231A460A21A04710BD10B538
:107080000A46846800230B21A04710BD10B5846810
:1070900000231A461021A04710BD10B544690023F3
:1070A000A04710BD0020704700230360074A82609C
:1070B000C2600261426180F8233080F8263083612B
:1070C000FF2380F8243080F828307047A570001026
:1070D000F8B504460F4616461D46FFF7E5FFA760C4
:1070E000E6602561069B63612046FFF7BAFFF8BDA5
:1070F0000423037000487047FC17002010B50A46AF
:10710000046900232021A04710BD10B5134604696F
:107110000A461721A04710BD00B583B08DF80710AF
:107120000DF107020121FFF7F0FF03B000BD0000E1
:10713000002301461A46184600F000B930B584070E
:107140008646034606D0A2B303F8011B980702F156
:10715000FF32F8D1032A26D95FFA81FC0F2A0CEB03
:107160000C2C0CEB0C402AD922F00F0C9C44C3E9E8
:107170000000C3E9020010336345F8D112F00C0F90
:1071800002F00F0517D04FEA950C1A460CF1FF34A8
:1071900003EB8C0C42F8040B6245FBD1043305F081
:1071A000030203EB840322B11A4403F8011B9A4241
:1071B000FBD1704630BD2A46002AF5D1F9E71546C5
:1071C000E1E700BF38B5074D074C2C1BA41005D0D4
:1071D000013C55F8043D9847002CF9D1BDE83840F2
:1071E00000F0F8B88474001084740010704700BF79
:1071F000704700BF844641EA000313F0030349D1FE
:10720000403A23D30B6803604B6843608B6883600C
:10721000CB68C3600B6903614B6943618B69836110
:10722000CB69C3610B6A03624B6A43628B6A8362F8
:10723000CB6AC3620B6B03634B6B43638B6B8363E0
:10724000CB6BC36340304031403ADBD230320BD39A
:107250000B6803604B6843608B688360CB68C360D6
:1072600010301031103AF3D20C3205D351F8043BF0
:1072700040F8043B043AF9D2043208D0D2071CBFCC
:1072800011F8013B00F8013B01D30B8803806046F5
:10729000704700BF082A13D38B07B1D010F0030347
:1072A000AED0C3F10403D21ADB071CBF11F8013BB7
:1072B00000F8013BA4D331F8023B20F8023B9FE7E2
:1072C000043AD9D3013A11F8013B00F8013BF9D255
:1072D0000B7803704B7843708B78837060467047EF
:1072E00020F0030110F00300C0F1000051F8043B4E
:1072F00000F1040C4FEACC0C6FF000021CBF22FA24
:107300000CF213434FF0010C4CEA0C2C4CEA0C4CE1
:10731000A3EB0C0222EA030212EACC1204BF51F8DA
:10732000043B0430F4D0C2F1000102EA0102B2FAD7
:1073300082F2C2F11F0200EBD2007047F0B51D4C83
:1073400083B00546164620681F460191FFF74EFFA1
:10735000194A019913682BB35A6820681F2A24DC44
:107360004DB9541C02325C6043F82210FFF740FF15
:10737000002003B0F0BD03EB820E0124022DCEF8F5
:10738000886004FA02F4D3F8886146EA040CC3F872
:1073900088C1CEF80871E4D1D3F88C512543C3F8E5
:1073A0008C51DEE7054B1360D6E7FFF721FF4FF066
:1073B000FF30DEE7FC0E0020AC100020B0100020F3
:1073C000024B13B10248FFF7B3BE70470000000044
:1073D000C5710010F8B500BF5FF800F0EF0600209F
:1073E0005FF800F0230200205FF800F0490700205A
:1073F0005FF800F0A50A00205FF800F07502002099
:107400005FF800F0F50500205FF800F0FD060020B1
:107410005FF800F0F10100205FF800F02106002085
:107420005FF800F0110100205FF800F0CD020020AD
:107430005FF800F04D0A00200119001079180010C3
:10744000A51800109D190010E11800101D1800105B
:1074500025190010E91700107D0B00102D190010E0
:10746000F51300106518001013190010C51800104E
:10747000F905001051060010C173001059370010B3
:0474800055020010A1
:10748800466F6F00426172000A2A2A2A2050414E34
:107498004943202A2A2A0A000A0000004E6F207356
:1074A80070696E6C6F636B732061726520617661C1
:1074B800696C61626C65000030783163203D3D2065
:1074C800282A696E7374293E3E3131750000000028
:1074D8002F7661722F686F6D652F76616C656E749B
:1074E800696E772F50726F6A656374732F43616C8E
:1074F80063756C61746F722F64656E74616368691B
:107508002D746573742D6669726D776172652F705D
:1075180069636F2D73646B2F7372632F7270325FA0
:10752800636F6D6D6F6E2F68617264776172655FEE
:107538006972712F6972712E6300000064656C7442
:1075480061203E3D202D32303438202626206465C7
:107558006C7461203C3D20323034362026262021B0
:107568002864656C74612026203129006375727265
:10757800656E74203D3D205F5F756E68616E646C5A
:1075880065645F757365725F697271207C7C2063C6
:10759800757272656E74203D3D2068616E646C651D
:1075A800720000006972715F68616E646C65725F79
:1075B800636861696E5F667265655F736C6F745F3F
:1075C80068656164203E3D20300000007674616289
:1075D8006C655F68616E646C6572203D3D205F5F1D
:1075E800756E68616E646C65645F757365725F69FA
:1075F80072710000212828282875696E74707472C9
:107608005F742972656D6F76655F7468756D625F0A
:1076180062697428767461626C655F68616E646C17
:1076280065722929202D20282875696E7470747256
:107638005F74296972715F68616E646C65725F63FB
:107648006861696E5F736C6F7473292920252073D4
:10765800697A656F662873747275637420697271CC
:107668005F68616E646C65725F636861696E5F73A1
:107678006C6F74292900000069735F736861726513
:10768800645F6972715F7261775F68616E646C656F
:107698007228736C6F745F68616E646C6572290020
:1076A800657863657074696F6E000000666F756E4B
:1076B800640000004E6F2075736572204952517343
:1076C8002061726520617661696C61626C65000099
:1076D80031203D3D202875696E747074725F74297D
:1076E8006C2D3E7370696E5F6C6F636B00000000F9
:1076F8002F7661722F686F6D652F76616C656E7479
:10770800696E772F50726F6A656374732F43616C6B
:1077180063756C61746F722F64656E7461636869F8
:107728002D746573742D6669726D776172652F703B
:1077380069636F2D73646B2F7372632F636F6D6D45
:107748006F6E2F7069636F5F73796E632F6D7574D9
:1077580065782E6300000000746F74616C0000008F
:107768006D74782D3E636F72652E7370696E5F6CF1
:107778006F636B006C6F636B5F69735F6F776E65C8
:10778800725F69645F76616C6964286D74782D3EF8
:107798006F776E65722900006D74782D3E656E7482
:1077A80065725F636F756E7400000000706F6F6CB8
:1077B8002D3E74696D65725F616C61726D5F6E7587
:1077C8006D203D3D2074696D65725F616C61726DFD
:1077D8005F6E756D000000002F7661722F686F6D07
:1077E800652F76616C656E74696E772F50726F6A5B
:1077F800656374732F43616C63756C61746F722F6A
:1078080064656E74616368692D746573742D666947
:10781800726D776172652F7069636F2D73646B2F5A
:107828007372632F636F6D6D6F6E2F7069636F5F17
:1078380074696D652F74696D652E63006465666192
:10784800756C745F616C61726D5F706F6F6C5F698E
:107858006E697469616C697A6564282900000000A2
:10786800417474656D7074656420746F20736C6501
:10787800657020696E73696465206F6620616E208B
:10788800657863657074696F6E2068616E646C6595
:10789800723B2075736520627573795F77616974CF
:1078A80020696620796F75206D757374000000007B
:1078B800486172647761726520616C61726D202520
:1078C8006420616C726561647920636C61696D65BF
:1078D8006400000076636F5F66726571203E3D202C
:1078E8005049434F5F504C4C5F56434F5F4D494E94
:1078F8005F465245515F485A2026262076636F5FBF
:1079080066726571203C3D205049434F5F504C4C96
:107918005F56434F5F4D41585F465245515F485A45
:10792800000000002F7661722F686F6D652F7661F9
:107938006C656E74696E772F50726F6A65637473C5
:107948002F43616C63756C61746F722F64656E741C
:10795800616368692D746573742D6669726D7761EA
:1079680072652F7069636F2D73646B2F7372632F49
:107978007270325F636F6D6D6F6E2F6861726477BE
:107988006172655F706C6C2F706C6C2E6300000008
:107998006662646976203E3D2031362026262066C0
:1079A80062646976203C3D203332300028706F7362
:1079B800745F64697631203E3D2031202626207090
:1079C8006F73745F64697631203C3D203729202627
:1079D800262028706F73745F64697632203E3D20DC
:1079E8003120262620706F73745F64697632203CDC
:1079F8003D203729000000007265665F6672657178
:107A0800203C3D202876636F5F66726571202F20C9
:107A1800313629004465627567000000626F6F7433
:107A2800325F77323571303830000000322E322E16
:107A3800300000007069636F3200000064656E7486
:107A480061636869000000004A616E2032302032AC
:107A580030323600666E692B00000000666E6900E1
:107A68006E616E00666E692D000000002C20667540
:107A78006E6374696F6E3A2000000000617373656D
:107A88007274696F6E2022257322206661696C65A5
:107A9800643A2066696C6520222573222C206C6963
:107AA8006E65202564257325730A000066616C7372
:107AB800650000002F7661722F686F6D652F766103
:107AC8006C656E74696E772F50726F6A6563747334
:107AD8002F43616C63756C61746F722F64656E748B
:107AE800616368692D746573742D6669726D776159
:107AF80072652F7069636F2D73646B2F7372632FB8
:107B08007270325F636F6D6D6F6E2F7069636F5F38
:107B1800737464696F5F7573622F737464696F5FE0
:107B28007573622E630000005553422073746469B4
:107B38006E202F207374646F757400005261737027
:107B48006265727279205069000000005069636FA5
:107B580000000000426F617264204344430000004B
:107B680052657365740000007263203D3D20340047
:107B78002F7661722F686F6D652F76616C656E74F4
:107B8800696E772F50726F6A656374732F43616CE7
:107B980063756C61746F722F64656E746163686974
:107BA8002D746573742D6669726D776172652F70B7
:107BB80069636F2D73646B2F7372632F7270325FFA
:107BC800636F6D6D6F6E2F7069636F5F756E69712E
:107BD80075655F69642F756E697175655F69642E77
:107BE800630000006C656E203E2030006E6578747E
:107BF8005F6275666665725F707472203C2075738B
:107C0800625F647072616D2D3E6570785F64617447
:107C180061202B2073697A656F66287573625F64CB
:107C28007072616D2D3E6570785F646174612900C2
:107C38002F7661722F686F6D652F76616C656E7433
:107C4800696E772F50726F6A656374732F43616C26
:107C580063756C61746F722F64656E7461636869B3
:107C68002D746573742D6669726D776172652F70F6
:107C780069636F2D73646B2F6C69622F74696E79F9
:107C88007573622F7372632F706F727461626C65A3
:107C98002F72617370626572727970692F727032B7
:107CA8003034302F6463645F7270323034302E6346
:107CB80000000000556E68616E646C65642049526E
:107CC8005120307825780A007268706F7274203DF0
:107CD8003D20300021286275665F6374726C20262F
:107CE800205553425F4255465F4354524C5F4655B8
:107CF8004C4C29002F7661722F686F6D652F766165
:107D08006C656E74696E772F50726F6A65637473F1
:107D18002F43616C63756C61746F722F64656E7448
:107D2800616368692D746573742D6669726D776116
:107D380072652F7069636F2D73646B2F6C69622F86
:107D480074696E797573622F7372632F706F7274B2
:107D580061626C652F7261737062657272797069A5
:107D68002F7270323034302F7270323034305F7589
:107D780073622E63000000006275665F6374726C44
:107D88002026205553425F4255465F4354524C5F6C
:107D980046554C4C000000006570202530325820B4
:107DA80077617320616C72656164792061766169BD
:107DB8006C61626C6500000043616E277420636F1C
:107DC8006E74696E75652078666572206F6E2069BD
:107DD8006E616374697665206570202530325800BD
:107DE8005741524E3A207374617274696E67206EFF
:107DF8006577207472616E73666572206F6E20619C
:107E08006C72656164792061637469766520657058
:107E180020253032580D0A0025732025643A204168
:107E28005353455254204641494C45440D0A0000DD
:107E38006972715F6164645F7461696C5F746F5FBC
:107E4800667265655F6C6973740000006D616B65CF
:107E58005F6A5F31360000007265736F6C76655F2C
:107E68006A5F3136000000006972715F6164645FA7
:107E78007368617265645F68616E646C6572000046
:107E88006972715F7365745F6578636C7573697621
:107E9800655F68616E646C65720000006D7574657D
:107EA800785F6578697400006D757465785F656ED4
:107EB8007465725F626C6F636B5F756E74696C007A
:107EC80072756E74696D655F696E69745F6D7574DE
:107ED80065780000616C61726D5F706F6F6C5F67D1
:107EE80065745F64656661756C740000616C6172CD
:107EF8006D5F706F6F6C5F6972715F68616E646CE3
:107F080065720000706C6C5F696E69740000000037
:107F180006005250D3F075421C7A001006005250E9
:107F2800E182887F247A001006005250ABB3605378
:107F3800347A001006005250BBFF3CB63C7A001061
:107F480006005250861C0302447A00100600525064
:107F58005422A29D507A001005005250DE65F46844
:107F68004CB1001000000000000000000000F03FCD
:107F780000000000000024400000000000005940FC
:107F88000000000000408F40000000000088C3404F
:107F980000000000006AF8400000000080842E41C4
:107FA80000000000D01263410000000084D7974110
:107FB8000000000065CDCD410D0A00000000000062
:107FC800A931001000000000AD310010B9310010D7
:107FD800F1310010ED310010000000000A0000002F
:107FE80000000306A6000800020002009C0014001E
:107FF800030057494E55534200000000000000009E
:10800800000080000400010028004400650076009C
:1080180069006300650049006E0074006500720025
:108028006600610063006500470055004900440090
:1080380000004E007B006200630037003300390007
:108048003800630031002D003700330063006400FE
:108058002D0034006300620037002D00390038001D
:10806800620038002D00390031003300610038000B
:1080780066006300610037006200660036007D001C
:1080880000000000050F2100011C100500DF60DD65
:10809800D88945C74C9CD2659D9E648A9F00000381
:1080A80006A60001000000000600525053B4F4A1D7
:1080B800307B0010737464696F5F7573625F696EFB
:1080C8006974000000000000447B0010547B00101D
:1080D800CC1E00205C7B0010687B00100902540055
:1080E800030100807D080B00020202000009040061
:1080F80000010202000405240020010524010001FA
:10810800042402060524060001070581030800105F
:1081180009040100020A00000007050202400000ED
:10812800070582024000000904020000FF00010563
:1081380012011002EF0201408A2E0900000101021B
:10814800030100007069636F5F6765745F756E692E
:108158007175655F626F6172645F69645F73747281
:10816800696E67005F72657472696576655F756EC2
:10817800697175655F69645F6F6E5F626F6F7400C8
:108188006463645F656470745F786665720000009C
:108198006463645F7365745F6164647265737300BC
:1081A8006463645F696E745F656E61626C6500002C
:1081B80068775F656E64706F696E745F616C6C6F11
:1081C800630000006463645F696E69740000000006
:1081D80073796E635F65705F6275666665720000CD
:1081E800757362645F656470745F786665720000B9
:1081F800757362645F656470745F6F70656E0000AC
:10820800757362645F6F70656E5F656470745F70CC
:108218006169720071756575655F6576656E740074
:1082280070726F636573735F6765745F64657363AA
:10823800726970746F72000070726F636573735F38
:108248007365745F636F6E666967000070726F6351
:108258006573735F636F6E74726F6C5F726571754F
:1082680065737400636F6E66696775726174696FB0
:108278006E5F7265736574007475645F7461736BA7
:108288005F657874000000007475645F7268706FD1
:1082980072745F696E69740000000000154F001069
:1082A800AD4F0010ED4F00106550001091510010B7
:1082B800B9520010000000000000000041540010F6
:1082C800D154001001550010455500104D320010D2
:1082D8008D56001000000000757362645F636F6E56
:1082E80074726F6C5F786665725F6362000000008D
:1082F8007475645F636F6E74726F6C5F78666572B5
:1083080000000000636463645F786665725F63629F
:1083180000000000636463645F6F70656E000000B6
:108328007475645F6364635F6E5F77726974655FB9
:10833800666C75736800000076656E646F72645FC2
:108348006F70656E0000000074755F656470745F1F
:1083580073747265616D5F726561645F786665727A
:108368000000000074755F656470745F73747265F3
:10837800616D5F77726974655F7866657200000089
:1083880074755F656470745F73747265616D5F772F
:10839800726974655F7A6C705F69665F6E65656443
:1083A8006564000074755F656470745F76616C69FC
:1083B8006461746500000000747573625F726870B0
:1083C8006F72745F696E69740000000092000202A7
:1083D8000304030504060B00FE08FE09FF01420220
:1083E8008407AB20050066072107C14367280122DF
:1083F800071B57275901230DBD42AF4C69A86AA82E
:10840800322500240DCD3E37AF4AE59D54B52300F3
:10841800250CC5422FAAEE8C726AC904260DC542E6
:108428002FA7987295648A510527071B574F950007
:10843800280A533F37C514DB3107290B533F27C799
:108448001C5B3145002A0AAD46AF8E43E694002BEB
:108458000AAD4637A3386446112C07A33ACF2A0140
:108468002D068C4E67042E06124367042F10D53E46
:108478001F659433CA19E58C724619013008C44245
:10848800CFE965013108C34237ADD803320AC44287
:1084980067C55CB64700330CC44267A39C34CA79ED
:1084A8002400340AC442375A5D23E604350BC4421B
:1084B80067E8BC51CE2301360BC4424FE5BCA299F4
:1084C8001400370AC44267E432C75C02380BC4425E
:1084D8004F459954349302390AC4424F4533ED4A03
:1084E800013A072A4367C4113B08BB3ACF465609ED
:1084F8003C0ABC423FB6514619053D089D4A67688B
:1085080038043E0BBC4227A38C328A6D003F0CC551
:10851800426FE58C724D671401400CC5425746B94D
:10852800924A526538410AC4424FAA28C7340342C6
:108538000BC44267453952344702430AC4424F4587
:10854800DD991400440AC44247A6D22B4900450AC3
:10855800C44267E8BC723D024609444367E8BC72FE
:108568001B470AC4424F455D4D99064809C4422736
:108578009A633A034908434367C55E034A09C442FC
:1085880057B7A54C0A4B0AC442275A49A64E194C5C
:1085980008C44227F73D024D0CC54227AF915652F9
:1085A80049DB014E0AC44227CAB5D429034F09C47E
:1085B800424F459F4901500AC442674573A45C0372
:1085C800510ACC3E4F45E772A300520AC4426745A0
:1085D80039524F19530CC4424F458D32CA482605AB
:1085E800540FC54267C88C32CA28A38C328A0055FA
:1085F80009C44227FA991400560BC54227BB539960
:10860800724611570CC54227BB924A6395290158F7
:108618000AC442279A49AA6806590EC54227EB544C
:10862800A69C51461945005A0BC44267E498638ECC
:1086380079045B08533F67C47E0E5C11D53E27A3BF
:108648000C33CA30A30C33CA30A3005D08533F670C
:10865800F673045E079D5637A73A5F068C42670497
:1086680060071B5747E600610AB4424FA334A24C87
:1086780003620AC44227E7159D23016309B4424FE8
:10868800455DA3016409C442BF1AD199066509B4BE
:10869800424FC5B1331A660AC44257E538526E02D2
:1086A800670BC43A6F447368391200680AC44227DA
:1086B800572349670069094B432F6624BB066A0A9A
:1086C8005C3ABFC6BA5B26056B0BC44227972AC91A
:1086D80054CA006C07434347F6356D0BB542E74A69
:1086E8002AA9A4922A6E09B442278D249D016F09F4
:1086F800B4424F45675200700AC43A6745E74839A3
:10870800037109C43A6F4467DA057208B44267A472
:108718007613730AB4426F648DF44800740AC44235
:108728002FC791721B097508B442277AA601760BE8
:10873800B54227EB54A69C5104770BB542275B49F9
:1087480055332500780AB44227CA24559401790B79
:10875800C43A279AA9D2314A007A09B44267E4D8C0
:108768001E017B0FD53E5F669451D41A66945186DC
:10877800027C06D13FE7117D0FD53E47C38C32CA34
:1087880050CB8C328A1A7E099D562FAA241300A03A
:10879800079D4227EB31A107C13B470D01A20AC43F
:1087A8003E378ED4CF9900A30BC5425756796794AC
:1087B800F318A40AAD4627A799E2CA01A50DC54238
:1087C80027EB540D1987CC2802A607D13F67C4119F
:1087D800A70ED43A4FC594559449A7981400A807F2
:1087E800135B27A900A90D4E3E57C794D4BE952AFE
:1087F800B304AA0AB44A4FA334464623AB08A54695
:108808002FCA141BAC079C4667E402AD050B4F67E3
:10881800AE0F4E3E57C794ACB4D2B2928A5902AF4B
:10882800068C5E6704B009A4524F45991400B10C38
:10883800BD4237A3386446991A02B208AC524FC5F4
:10884800E608B30AAC5267A3A4D14800B4071B5783
:10885800379500B50AC43A277A8DA43300B60EC5F9
:10886800426FA8A42A15534C31C514B706124B679A
:1088780004B809A43A3767341200B9062A536F3589
:10888800BA0AB44A4F4599341C01BB09A54627B614
:10889800A24C00BC0ED53A2F6B1453A953A5E5C8BA
:1088A80009BD0DD53A2F6B1453A95337CA79BE0E9B
:1088B800D53A47C31CA3DAA9D272E404BF0BC53A60
:1088C80037A34CB7514E0BC00BCC422FA368C53110
:1088D800CD00C10ACC42B7962A8E6906C20BCC429B
:1088E800B74A52C531CD00C30BCC422FA968C53158
:1088F800CD00C40ECD4247696C5623C514534C00B5
:10890800C50BCC424FC524551CD30CC60EC5426FAF
:108918002499621A33C514D300C70BD43A4F45DDE6
:1089280099748C00C80CCC422FA334745E398F0024
:10893800C90BCC42B71C3AAF9C4700CA0BCC42B714
:108948001A3BAF9C4700CB0FCD42476938524619B6
:10895800CD8C321A09CC094B4327A715BB06CD0984
:108968004B4337A515BB06CE094B43AF1A29760DE5
:10897800CF0ECD424769BC33CA28A38CF202D00D72
:1089880045424FA718472A534CA504D10BCC422F78
:10899800A9722D75CA00D20BCC422FA3A8A2675288
:1089A80000D30ACC42B756D1332900D40ACC42B7F7
:1089B8004A2A7A2605D50BCC422FA9A8A2675200CD
:1089C800D60ECD4247692CAB98628A294609D70949
:1089D800AD4627A7BAAA03D80F563E1FC6D9924953
:1089E800AAA862393304D90ACC422FA3D26752000D
:1089F800DA09CC42B7E9332900DB0ACC42B7CA28E6
:108A08007A2605DC0FCD42476958C514534C31C549
:108A18002801DD0DCD42BFCC3AD51965945104DE4D
:108A28000BC44227E715E5483903DF09C4424F451F
:108A3800D5E912E00CCC422FA38C354A23CA34E185
:108A48000BCC42B7A6344A23CA34E20CCC42B7CA8C
:108A580050A334A24C03E30CCC422FA98C354A23F3
:108A6800CA34E40BCC42AF1B6A94469469E50CCC3B
:108A780042B78A51A334A24C03E60CB54247C994C5
:108A8800868A292A01E70AC43A4F455DA35902E8B4
:108A98000CCC422FA38C551C3BA301E90BCC42B74D
:108AA800A6541C3BA301EA0BCC42B7CA50C5B1334C
:108AB8001AEB0BCC42AF1BAA38764603EC094B43A2
:108AC800276724BB06ED084B43AF86B26BEE084B15
:108AD80043AF2DBB06EF094B4327A92CBB06F00C6F
:108AE800C44227258D6292665200F10BCC422FA911
:108AF8000CD348D219F20BCC422FA38C55742605FF
:108B0800F30ACC42B7A654742605F40BCC42B7CA74
:108B18005045675200F50BCC422FA98C5574260599
:108B2800F60ACC42AF1BAAE84C0AF70CBD4237A3A1
:108B38004C0D4D651401F80D463E1FC6D9922A9674
:108B4800334300F90ACC422FA30CA3671AFA09CCC5
:108B580042B7C6D1330DFB0ACC42B7CA287AA60160
:108B6800FC09CC42AF1B45CF34FD0CDC3AB7C6D16B
:108B78004C958E5102FE0BD43A2757C9944BD51900
:108B8800FF0CDC3AAF1B4533553A4609000000108C
:108B9800016404DC01C90512022E0539FFFF01003A
:108BA8000CCC42676468C531CD0001010CC4426F2A
:108BB800438DD288320D01020CCC42272669C5317B
:108BC800CD0001030DCC4227268D354A23CA340136
:108BD800040CD43A4FAA28C7346B1401050DC43AC3
:108BE8004FA334A24C33A30001060BCC42B7565115
:108BF80037930201070CCC423F66ACA2AED100010C
:108C0800080CCC42B74A2AEA66520001090CCC4249
:108C1800B7CA50455DA301010A0CCC424F631575D4
:108C2800332900010B0CCC423767ACA2AED100014E
:108C38000C0CCC42AF8C2AEA665200010D0CCC42D7
:108C4800AFCC58455DA301010E0CCC4227C5285373
:108C5800E94A12010F0FCD425FA668A698628A29D9
:108C68004B0001100E45424FA718472A534CA50444
:108C780001110EC5423F8E1C574C31C5B800011278
:108C88000DCC42676434745E398F0001130BC44203
:108C98006F4315C7CE6801140DCC42272635745E84
:108CA800398F0001150DCC4227268D551C3BA30199
:108CB80001160CCC424FC3A1F3CA790401170CCC9E
:108CC800423767ACE2D8190D01180DD43A67E8BCF1
:108CD800723D62460101190CC43A4FC5B1339A1965
:108CE80005011A0CCC42AF4C43E795F308011B0C65
:108CF800CC42AFCC58C5B1331A011C0CCC42B74A90
:108D08002AEA34651A011D0EDC3AB7CA7044736842
:108D1800391200011E0DCC422726A9A24E53A601E6
:108D2800011F0EDC3A27268D473487962301012040
:108D38000CCC424F6315759A320D01210DDC3A3780
:108D4800673CA239B41C0901220CD43A4F455D4D49
:108D580099660901230CD43AB71ED11C5A8E040116
:108D6800240CCC42B7CA28CA31CD0001250CCC420C
:108D78002FA6BA1A499A0101260BC44227CA31C73D
:108D8800340301270E45422F8F9851B2CA14530C51
:108D980001280BCC422FA93873E70001290BCC42DC
:108DA8002FA98C75E700012A0BCC4267643873E75A
:108DB80000012B09434367CBAE01012C0BCC4227A2
:108DC800263973E700012D0BCC4227268D75E70065
:108DD800012E0A533B67C55E2B07012F0B5B3B2F08
:108DE8006624BB560E0130094B434FAFD8350131CD
:108DF80008334347760D01320AD43A27FA992B05EE
:108E080001330DDC3A27CA8CA2CF9C140001340C24
:108E1800CC42B78ABA963229000135115D3ABFCAE9
:108E28009446196594514665940001360DD43A2745
:108E38005A49A64E99620601370ED43A27972AC98D
:108E480054CA14330001380AB442275A6945190133
:108E5800390ACC423FA6DC7B04013A094B43AF9464
:108E6800BD06013B0AD43A27F73D6209013C0A5383
:108E78003B47F6B54A00013D0ACC4277AABA7B04C3
:108E8800013E0FCD427FC4546694514619E509014D
:108E98003F0FC54227A38C32CA36CA682400014056
:108EA8000FC54247A38C328A29A68CF20401410ED1
:108EB800C5422FA38C4A1B6594D10801420A43433B
:108EC800479623560301430BCC42B7B9963A65003F
:108ED80001440BCC42B7C66924E90C01450DD43ACC
:108EE80027CAB5D42953CC0001460CC43A278D248F
:108EF8009D29660001470CCC4227C5722D75CA0012
:108F080001480CCC42AFCC308D249D0101490F4D56
:108F18004247A39C61B2CA14534C31014A0CD43A5B
:108F2800278D247DE6A400014B0CC43A278D249D8F
:108F3800392900014C0CCC426764A8A26752000191
:108F48004D0BC4426F43159D4901014E0CCC42277D
:108F580026A9A2675200014F0CCC4227268D5574D2
:108F6800260501500FCD422FCA28AB98628A2946A0
:108F78000901510FCD422FCA4CC92AA69862940004
:108F880001520FC5426FA898621A29A698F20801E3
:108F9800530DB5426FA8A4468A298F0001540CCC02
:108FA80042B75C518ED4940101550BCC42B7C6230D
:108FB800B59B0001560DD43A674539524F99620660
:108FC80001570BC43A67A4761BC50801580DCC425B
:108FD80027C5B8A21CA9290301590BCC42AFCC70F4
:108FE800A47613015A0DCC42B75651238D64520012
:108FF800015B0DCC423F663CB2467A2400015C0D11
:10900800CC42B74A2A6AA4914C0A015D0DCC42B7FA
:10901800CA70648DF44800015E0FD43A4F458D3212
:10902800CA48261D2300015F0CC43A6F648DF4C83A
:10903800310201600DCC42AF8C2A6AA4914C0A011E
:10904800610DCC42AFCC78648DF44800016212D532
:109058003A67C88C32CA28A38C32CA3047000163E9
:109068000CD43A2FC791721BC912016410CD42AFBC
:109078008E436694514619651401016510CD425F0F
:10908800C5548D9851461965A80001660FC54267F9
:10909800C88CF2CE28A38C220001670DC4422FC7CA
:1090A80091E24839230101680CCC422FA90CA3672F
:1090B800520001690BCC422FA90CA3671A016A0B55
:1090C800CC426764147D2605016B0AC4426FA3E88D
:1090D8009906016C0CCC4227260DA3675200016D3E
:1090E8000BCC4227260DA3671A016E0BCC42B78A18
:1090F800297A2605016F0BCC42B78A297AA6010185
:109108007010CD422FCA8C638A29A69862940001F8
:109118007110CD422FCA8C638A29A698625C00011F
:10912800720BD43A27FA9974460101730BC43A2793
:109138007AA699510001740ECD4237A7DA4A2A8DD2
:1091480055A60401750ECD4237A78CB395543553F7
:109158000201760FCD4237A75AA73AA38C328A006C
:1091680001770EDC3AB7CA289AA9D2314A000178A9
:109178000FCD4247699875AA33CA28A30801790C0C
:10918800CC42B71C39D6318F00017A0BCC42B7C616
:1091980023C7F608017B0CCC424FC391631DF3082B
:1091A800017C0CCC42376738726C8F00017D0CCC87
:1091B80042AF4C23C73AE611017E0CCC42AFCC70CB
:1091C800E4D81E01017F0943436FC99E0001800E48
:1091D80045422F8F98D1AC628A690101810EC54240
:1091E8006F552AD929A698A20201820CC44267E5C4
:1091F800BCA239120001830BC44267E5159D230107
:1092080001840EC5422F6B94D1AC628A6901018535
:109218000AB4422F6A995A0A01860BC4424FC5DC28
:1092280096490101870FCD425FC92AA38C32CA280B
:10923800460901880DC5425F6659659451860B0140
:10924800890E45424FA718472A534CA504018A0F97
:10925800C5426F552AA932C514535400018B0AC45C
:10926800426F57239A69018C0AC4426FA7119D69FE
:10927800018D0CC43A4F4533E98C4602018E0AC46D
:109288004267E46AD743018F0CC4424FC59CC79418
:10929800490101900CC4424F458D542E930201910F
:1092A8000FC5426FA48C329A19659D110001921066
:1092B800553A5F669447CC28A38C328A1A01930FDB
:1092C800CD425FC92AA38C928A29C60501940FD57D
:1092D8003A27DBA94C39A39C62CA11019510C542F3
:1092E80027A38C964A2AA9A4924C0001960BC44243
:1092F80047E64E99140001970A434367C5B462359F
:1093080001980FC54227A64A459D628A554C00011F
:10931800990CC4424FE5A8924CA50C019A0A434304
:1093280047562B5603019B0BC4422F233BAA6806C2
:10933800019C10C54227259554524925955435025C
:10934800019D0FC5422FA6985452954A23EA000161
:109358009E0BC43A278D249DB900019F0CC4424F2F
:109368004539A699140001A010CD421F2533C51414
:10937800534C31C5280101A10DBD421F2533C51429
:10938800538C1201A211D53ACF1A29A9A4924AAA3C
:109398009951460101A30EC53ACF1A29A9A49A19D1
:1093A800651401A40EC5426F552AA9526794510449
:1093B80001A50CD43A4FE5159D23E50C01A60CCC6C
:1093C8003E27AF2847EA990301A70CC4424FC51CA2
:1093D800DB31290001A80BB44267A33862460301B8
:1093E800A90CC442676894518EF50801AA11D53AB0
:1093F8002FA7AC51461965945146190A01AB0DD4F3
:109408003A2FC791721BE9A40001AC10C5426FA89E
:109418009832CA28A38C328A0001AD0BC44257C5C2
:1094280091721B0901AE0FC54267C88C32CA28A3C6
:109438008C321401AF10CD421FC999628A29A698AF
:1094480062940001B00DBD421FC999628A29C60500
:1094580001B10BC54247A9B6775A0001B20AC44206
:109468002795BE620401B30FC54227A64AB55146E7
:109478001965940101B40FD53A1FE599628A516BB9
:1094880094B30601B50DC44267E49846CA318F000B
:1094980001B60BB44267C43452CC2301B70DC442A1
:1094A80067E41835CA32290001B80CC442676894C9
:1094B800552E930201B90CC43A676894552E93024D
:1094C80001BA0DC43A67E418354A2A230501BB0DD1
:1094D800C44267C51CD348318F0001BC0DC4426724
:1094E800A4AC51CE72240001BD0BB44267A4AC51A8
:1094F8001E0901BE0CC44237C7995196490101BFE4
:109508000CC43A2725D34A32670001C007D13BE78C
:109518001101C109533B27F9AF0001C211D53A37F0
:10952800A38CE29071C88C32CA280201C308C143D7
:1095380067280101C40ECD4237ADA45652C94A5618
:109548003201C50ECD4237ADA4D348492557320163
:10955800C60FCD4237459D874A2A59498E0001C713
:109568000CC542276EAFA4D2500001C80FDD3A1FC8
:10957800698DE2768F9451540001C9135D3A1FCD6D
:1095880094515231C514531C29A3A80001CA10C50F
:1095980042278D94461A69249554B20001CB12DDF6
:1095A8003A1FA9A4E21A6924955452358A0A01CCB3
:1095B80012DD3A1F6594A1955452492555A3A80078
:1095C80001CD0BCC42AF8C561CD30C01CE0DCC4236
:1095D800AFCC58A334A24C0301CF0A4B4327552BD9
:1095E800760D01D00A4B4327D548760D01D10BCC17
:1095F80042AF8C2A7A260501D20CCC42AFCC584512
:1096080067520001D30BCC42AF4CD167520001D452
:109618000BCC42AFCC307AA60101D50CCC4267A462
:109628001A45CFA40001D60FCD426764AC34AC62B2
:109638008A29C60501D70CCC42278D9451F44C0ACF
:1096480001D80FCD423767A56115534C312E000163
:10965800D90FCD4247AD1A5631C514538C1201DAD1
:109668000FCD42AF8E4AC32AA698625C0001DB0B7D
:10967800CC4247D9287A260501DC0FCD4237C3648E
:10968800C32AA698625C0001DD0BB44267A33C665E
:10969800520001DE0CCC4267A41A5A714C1901DF42
:1096A8000FCD426764AC34D630AE18170001E00D18
:1096B800CC426764A8B18A63CA0001E10DCC426755
:1096C80064A8B14669C43401E20FCD4267646A24D4
:1096D80099E25831C53401E30EC5426F6325531A28
:1096E8002AA6A80401E40FC5424F56196594541AD6
:1096F800312E0001E50FC53A6FC514534C238F98DE
:10970800260001E60CCC42AF8C2AEA34651A01E740
:109718000EDC3AAFCC7844736839120001E80CCCFF
:109728004227C5D24A32953201E90DCC422FA93AD7
:10973800AA2453290301EA0BD43A4F459F496714D9
:1097480001EB0BC43A4F4567D2190501EC0DDC3A21
:109758006764A8A267D2190501ED0CD43A6F4315C6
:109768009D49671401EE0DCC42AF4C23C7A8914C1C
:109778000A01EF0FDC3AAFCC70E41835CA32290081
:1097880001F0115D3A37E54C6A9451461965544623
:109798000901F10EC542478DA8924A56B2920101BD
:1097A800F20DC54247EB345252C9950C01F30EC570
:1097B8004237A33C5452C94A720401F40CCC42B754
:1097C8005651A729D30001F50DDC3AB7A6463487D0
:1097D80096230101F610C54227C514531A49259549
:1097E80054920901F70CC44227255325996B0001AF
:1097F800F80CCC422FA3722D75CA0001F90CCC428B
:109808002FA30CD348D21901FA0DCC4257A998A41A
:109818008A63CA0001FB0DCC4257C514B34669C41C
:109828003401FC0ECD42BF1E49A638564C310D01FD
:10983800FD0ECD42BFA6CC94868A292A0101FE10CE
:10984800563E3FA318674BAAA86239330401FF109C
:10985800563E3FA34CC6D9922A9633430002000EC7
:109868004D422736B5AC468A29A61802010E4D424C
:1098780027B6290DE38A29C60102020CCC424FC53E
:1098880024551CD30C02030DCC424FC50C354A237A
:10989800CA3402040F4D4227B646CA28A399514636
:1098A8002302050E4D4227B629598D94518603028D
:1098B800060CCC424FC5B1F3CA790402070DCC425D
:1098C8004FC50C551C3BA30102080E4D42273677A5
:1098D80046196594511E02090E4D4227B6298D324C
:1098E800CA28A33C020A0BCC424FC53473E70002D6
:1098F8000B0BCC424FC50C75E700020C0F4D4227ED
:10990800366515534C31C5A800020D0E4D4227B6D9
:109918002959C514538C0A020E0CCC424FC5A4A277
:10992800675200020F0CCC424FC50C557426050235
:10993800100E4D4227B66615D34CB18A0102110F9D
:109948004D4227B6F18829669451461102120DCC72
:10995800424FC591A21CA9290302130CCC424FC542
:109968008C466A37010214104D4227B6628A29A62E
:1099780098628A510102150F4D4227B6714C31C5C4
:1099880014538C0302160CCC424FC58CA2675200AC
:1099980002170BCC424FC58CA2671A02180FD43A93
:1099A8004F458D32CA48261D230002190CC43A6F50
:1099B800648DF4C83102021A12D53A67C88C32CACB
:1099C80028A38C32CA304700021B0CD43A2FC79107
:1099D800721BC912021C0DC44267A31835CA496517
:1099E80000021D0DC43A67A31835CA496500021E56
:1099F8000CCC42AFCC30CA31CD00021F0CCC422770
:109A0800C5BA1A499A0102200BD43A278D247DE65B
:109A180002022110CD3E37A32C534C31C5B4924ECF
:109A28000002220CC4422F49995434930202230D98
:109A3800C4422F4999A48A32290002240ED43A67D5
:109A4800E498638E79A3980002250CC43A67E4D899
:109A5800DE28260002260CCC424F63A9E298660055
:109A680002270DCC423767AC511A51A60102280CC7
:109A7800D43A67E8BC723D620902290CC43A4FC562
:109A8800B1339A2500022A0CCC4267A44A45CFA4D8
:109A980000022B0FCD426764AC3496554C314A0016
:109AA800022C0DCC4267A4A4A28ACEA400022D0DDC
:109AB800CC4267A4A43256D14C0A022E0BCC424F9A
:109AC80063153D9302022F0CCC423767ACA23329B1
:109AD8000002300CCC4267C41C5574260502310DB7
:109AE800CC426764A8B18A66520002320FCD426741
:109AF800689875AA33CA28A30802330DD43A6FA30D
:109B080068A64AC72801023411CD3E47A38C32CA41
:109B180028A38CD218310202350EBD3E67A6986282
:109B28008A69449D00023610CD3E2FA33C62461937
:109B38006594E48C0002370A443A5777CBA40002B4
:109B4800380EC54237A3BC2A955452D50202390EA5
:109B5800C53A6F552AA9A4AA9D5104023A11CD3ECF
:109B68004FA515535223A9A4CA941100023B0DCC4A
:109B78003E6F44D54BAAA43200023C0CC43E3FA918
:109B8800B492D42303023D0FC5422FA38CF2881947
:109B98006594D108023E0FCD3E67C814B5CE28CBD8
:109BA800143302023F0CC43A6F648DF48819090219
:109BB800400CC43A67E4D8CE28230102410BC442C2
:109BC8004FC51C656E0102420BB4424FC51C654E61
:109BD8000002430E45426F5631CD385299160002A5
:109BE800440FC54227A698621A33C514A304024538
:109BF8000CC54237A39C62AADD0102460DCC3E6724
:109C080048955625E5D00002470CC43E3FA9348646
:109C1800D4230302480FC54257A38CE2C829A618CB
:109C280025000249115D3A3FA34C6A94511C39A39F
:109C3800324A00024A12D53A6FC514534C31C594C2
:109C480064CA28C300024B0FC53A6FC514534C3180
:109C58006E946100024C0D45426F56D550658A5589
:109C68000C024D0BB44267A4E6483902024E0EC5F9
:109C78004227EBB1EA8C32CA2802024F0EC53A27B6
:109C8800A698862A35CA590302500C354267C42A59
:109C9800A699A10202510DB5426FC514534C31AAC1
:109CA8000002520D354227C92AA698625A0002536B
:109CB8000BC4424FE5159D230102540AB4424FC517
:109CC8005C8F0402550BBC3E4F455DA91501025639
:109CD80010D53A3FA3B8628A29A61837CA30025766
:109CE8000EC5425F6699628A29A62C0102580BB4F8
:109CF800424FC5A1F3480002590BB44267A33C6622
:109D08005200025A0BB54267433D568C12025B0B58
:109D1800B4426F64A4724603025C0BB44267A3A406
:109D2800511E09025D0CB5426743A57246690202DD
:109D38005E0BB5426F65A5B24E0B025F0BC43A3796
:109D4800B746CC4902026010D53A5F6699628A2903
:109D58006E1453D40002610CC43A6F44736839120C
:109D68000002620AB4426FE434651A02630EC53A0F
:109D780027EB546794534C390202640CB54247AD43
:109D880032A798720402650AC43A277AA9BA00026F
:109D9800660BC4424FE53492740602670DD43A4FFD
:109DA800E5349274E6A40002680B4B432F6624D373
:109DB8008A69026908334327760B026A09334367C5
:109DC800C5D600026B0DC5424FA38CB2B233CA0B85
:109DD800026C0DC5424FA32C53B533CA0B026D0953
:109DE800543B47F73712026E12553A47A38C468AFE
:109DF800A94C318E94515A00026F0DB54227259512
:109E08005452495523027010C53A27259554524992
:109E18005523A38C0202710FC53AE74A2AA9A492D6
:109E2800AA51540002720F453A2F59658A29A698FB
:109E380072460002730FC53A2759658A29A69851B8
:109E4800860102740AB44227AEA5CE0002750BB48F
:109E5800424FC53165520002760DB5426FA898464B
:109E68008A298F0002770CBD426F652BA9A4BA001E
:109E7800027810D53A37A3BC2A955452D5CE280279
:109E8800027909B44237B7AA11027A0AC44237F7ED
:109E9800AA4600027B0FC53A37A38C328A296E94F2
:109EA800A100027C0AC43A67A4764F00027D0AC466
:109EB8003A67A4763712027E09B4424F45BB0602C0
:109EC8007F09B4424F45991B02800BB4426745395C
:109ED80052940102810BB44227CA91A21C09028242
:109EE8000DC43A6F648DF448192900028311D53ADC
:109EF8005F6694514619659451465103028410D502
:109F08003A5F6694514619C591338A1A02850DB590
:109F18004247C38C32CA284301028610D53A5F668D
:109F280094514619659457350302870CC43A47A3E0
:109F3800DC1A31270002880BD43A2FC791726F249C
:109F480002890DB54227A698C64C312E00028A0B0D
:109F5800B54247A9B69D1600028B0AB4422795CE92
:109F6800A400028C0CB54237A39C62AA7500028D2E
:109F78000BB542AF5C954A5A07028E0AC44257D6BF
:109F8800AA6906028F0CB54227EB54679451040264
:109F9800900EC53A676494DB686494610002910B83
:109FA800BC3E67E4D81A2B0202920DC43A67E41843
:109FB80035CA32290002930DC43A67E41835AA5409
:109FC800520102940BC4424FC55CE6160002950B81
:109FD800C4424F459D516E0202960BC44237B75199
:109FE80096490102970AC43A4F45DD8D0602980C3E
:109FF800B5426F659554D2690102990BB44267C5A1
:10A0080091A21C09029A0BB5426FE564EBB40002F9
:10A018009B0EC5425FE695515231C5B800029C0AB5
:10A02800B44227CA31CD00029D11DD3A37A34C6AEC
:10A0380094514619E5A1A206029E0CC43A27CA54B7
:10A04800AA247301029F09B44227778F0002A01047
:10A05800D53A5F6699628A29A6AC51461102A10CCD
:10A06800C4424FC55CC699130002A20CC4424F45B6
:10A078009D519C390202A30EC54237A33C5452C9D4
:10A088004A720402A410D53A37A33C5452C96AA9AB
:10A098008CD20202A50FD53A37A33C5452C94A477D
:10A0A8002E0102A60F46422FC38C96AA93CC29C72D
:10A0B8000502A70E563A2FA79856ECEF0DB30402E7
:10A0C800A811563A2FC38C96EA9D72AA6C94510433
:10A0D80002A90F563A37A30CD318A9FF37CC0A02A6
:10A0E800AA0E454247A38C929D6215870202AB0FC8
:10A0F800454247A38C468AA94C510E0102AC0EC5B5
:10A108004227AB6AA65A5533250002AD0CC44267F4
:10A118004899C921650002AE10453A27A798628A76
:10A1280029C99451460102AF0D463A27C77EE994E2
:10A1380061C60102B00A2B5327C691540002B10927
:10A148002B536F8EA40202B20AB34E37231917009D
:10A1580002B308235367C41202B4082353B71C017F
:10A1680002B508AC4E37575B02B609235327AD3406
:10A178000202B70AA55227ABCE940002B80A2B4FA9
:10A1880027A932450002B9081A572F290002BA092F
:10A198009C56AFA5120002BB071A57CF0002BC0895
:10A1A8001A5747290002BD071A5767061E9E0DC594
:10A1B800426FC854A658654B0120800AAC3E4FA593
:10A1C8002993022081072A3F6F35208209AC3E4F30
:10A1D800C5E60820830BAC3E67A3A4D148002084C1
:10A1E8000AAC3E37AA6AC40420850AAC3E67E58DEE
:10A1F800460220860AAC3E4FE515930220870AAC3A
:10A208003E67E458470020880BAC3E4FC5A4625215
:10A218000020890AAC3E4FC5B4930220AC0CBD4265
:10A2280077E511F388190E2103114E422FA34A3501
:10A2380033CC30C38C5346022109114E422FA3342C
:10A24800928619EE0C33CC3003FB000C4642B78AD9
:10A25800ADB162BF00FB010E4E421FE51433AC8660
:10A26800ECD700FB020B46427776ADD8AF01FB0373
:10A278000E4E421FC691EA94C648FD1FFB040C46C9
:10A288004277A45E43F5FF00FB050FC5424F5669B0
:10A29800C414534C314501FB060EC5423FA3386434
:10A2A8008A554CA500000000416C0010B76C0010E6
:10A2B800DD6C00101815E215AE154015A115C01576
:10A2C800A615A2152F15F8160015231581161F15AA
:10A2D800AE15A519FF000000000196320101327881
:10A2E80000093D00000428501104000084002000EB
:10A2F8001815A015C819FF001815A115C019FF00D9
:10A308001815AE15A519FF001815A415AF19FF00EB
:08A31800DCCEFF7F0100000014
:10A32000187F0010247F0010307F00103C7F001049
:10A33000487F0010547F0010607F0010B080001034
:10A3400000B503460068EFF3108272B6D0E8CFEF95
:10A350005FF0010CBEF1000FF8D1C0E84ECFBEF1A6
:10A36000000FF3D1BFF35F8F93F90400002809DBDE
:10A3700079B10860002019680023C1E88F3F82F39B
:10A38000108800BD4FF0504191F900101971012063
:10A39000F1E70846EFE70000F8B51E460368002B1A
:10A3A00028D0044615464FF0504393F900301F461D
:10A3B0002168EFF3108C72B6D1E8CF2F0123002A69
:10A3C000FAD1C1E8423F002AF6D1BFF35F8F94F97A
:10A3D00004E0BEF1000F13DB22680023C2E88F3FC8
:10A3E0008CF310882846314600F032FE0028DFD07A
:10A3F00000200DE0074B084AA621084800F044FE63
:10A40000277122680023C2E88F3F8CF31088012057
:10A41000F8BD00BF68770010B07E0010F87600101D
:10A4200070B582B0064615461C4601A9FFF788FFA5
:10A4300038B99DF904204FF0504393F900309A4207
:10A4400001D102B070BD2A4623463046FFF7A4FF73
:10A45000F7E738B505460C4600F00AFEE30E4FEA72
:10A46000441CBCEB040C63F100039B0043EA9C73A7
:10A470004FEA8C0C1CEB040C43F10003DB0043EAB5
:10A480005C734FEACC0C10EB0C0243EB0103002B86
:10A4900003DB2846FFF780FF38BD4FF0FF326FF037
:10A4A0000043F6E708B50268EFF3108372B6D2E80E
:10A4B000CFCF0121BCF1000FF9D1C2E84C1FBCF194
:10A4C000000FF4D1BFF35F8F90F90420002A09DB5D
:10A4D000FF22027101680022C1E88F2F83F31088E8
:10A4E00040BF08BD024B034AD521034800F0CCFD14
:10A4F0007C770010A47E0010F876001008B50023C9
:10A5000008E00A4A0133002142F8331002EBC3028B
:10A510005160DBB20E2BF4D94FF470720021044865
:10A5200000F092FD034B044A1A6008BD0000105071
:10A53000C81A00208C1E0020800110502DE9F04325
:10A5400085B01F4B9E6D0024012504E026EA050618
:10A550006D000134E4B286B31F2C2ED82E42F7D002
:10A56000184B9D654FEA540904F0010787F0010775
:10A5700004F0FE033B44144A02EB4318404600F04B
:10A5800033FA0028E2D007EB49070F4B03EB4713E0
:10A590009978DA8A00238DF8043007208DF80500B9
:10A5A0008DF8081003928DF80930012101A800F000
:10A5B00039FA404600F0B3F9C8E705B0BDE8F083CA
:10A5C0000000115000301150881A00202DE9F0438E
:10A5D00085B0744BD3F8985015F4003647D0724BC1
:10A5E0009A6A724B1A60002427460AE0704B03EB0C
:10A5F0008413002283F83C2000F0BEF93746013472
:10A60000E4B20F2C19D8A20102F12000684B1844C3
:10A61000134493F83B30022BF1D1654B03EB8413C9
:10A6200093F83A60002EEAD0614B03EB841393F861
:10A630003C30002BDAD13746E1E73FB95D4B1B7860
:10A6400023B95D4B4FF40032C3F89020554B9B6CFF
:10A65000C3F30A0300228DF8042003228DF805209D
:10A660000293012101A800F0DDF94FF4003615F046
:10A67000100F06D115F4803F49D046F480360024EF
:10A6800023E046F01006FFF759FFF3E74FF002080A
:10A690004A4BC3F86080434B5B6E38EA0303FAD140
:10A6A0004FF440520021384600F040F9384600F09F
:10A6B00036F9414BC3F86480C3F860803C4B03EB30
:10A6C00049130122DA701444E4B2012C0BD8A146DC
:10A6D000374F07EB4417BB7E002BEFD0002CD5D0B3
:10A6E0004FF00108D4E700238DF8043006238DF8DD
:10A6F0000530334B93E8030004AB03E90300012169
:10A7000001A800F08FF92C4B4FF400321A6515F4B4
:10A71000805F0AD115F4804F1DD115F4004F2BD165
:10A72000AE423AD105B0BDE8F08346F4805600242D
:10A730001C4B1C60FFF7E2FE8DF8044001218DF8F0
:10A7400005108DF8084001A800F06CF91A4B4FF481
:10A7500000221A65DEE746F4804600238DF80430B7
:10A7600004238DF8053001210DEB030000F05AF9A8
:10A77000114B10221A65D0E746F4004600238DF8ED
:10A78000043005238DF80530012101A800F04AF9B5
:10A79000094B4FF400621A65C2E786EA05010948D1
:10A7A00000F06AFC0000115000000B40801A0020ED
:10A7B000881A0020DE1E00200030115000201150A9
:10A7C00000001050BC7C0010F8B504460F46838A88
:10A7D000068B9E4228BF1E469B1B838246F48062E6
:10A7E000C3787BB14FF40055154383F00103E37048
:10A7F00063784BB1A38A0BB945F4804507B12D04AA
:10A800002846F8BD1D46EFE7E0683246216900EBB7
:10A81000871000F029FC23693344236145F4004587
:10A82000E8E70000094B1B6C13F0020F0BD1837893
:10A83000DB0901D100207047C37E022B01D000202C
:10A840007047012070470020704700BF0000115082
:10A8500008B5FFF7E7FF40B1054B9B6A054A126850
:10A860009B1AA3F54873C62B00D808BD0020FCE74F
:10A8700000000B40801A002038B5044683681B682E
:10A88000084601B11B0CC3F30905627892B913F4B1
:10A89000004F09D1E38A2B44E382238BAB4201D9D9
:10A8A0000023A382284638BD0E4B0F4AE8210F48EB
:10A8B00000F0EAFB13F4004F0DD0E1682A4601EBEB
:10A8C0008011206900F0D0FBE38A2B44E3822369E6
:10A8D0002B442361E1E7064B034AEE21034800F0D5
:10A8E000D3FB00BFDC7C0010D8810010FC7C001082
:10A8F000807D001010B5044683681B680021FFF7B7
:10A90000BBFF63681B6813F0804F02D0238B834228
:10A9100000D010BD01212046FFF7AEFFF9E700236C
:10A9200083768382C38203617047000008B50B46BB
:10A9300011B1816809680B409AB1134312F4806F1A
:10A940000FD08268116811F4806F0DD123F48061FB
:10A950001160074A126C12F0020F02D10C22033A66
:10A96000FDD28268136008BD8178024800F084FB44
:10A9700000001150A07D001070B5044643681D68AA
:10A980000021FFF721FF40F48056164B1B6C13F09B
:10A99000020F13D0A37813F07F0F14D10023A28AE3
:10A9A00002B1A3B125F0A04545F0005563681D60D4
:10A9B000324600212046FFF7B9FF70BDA378DB09BE
:10A9C00003D10123EBE70123E9E70023E7E70121B6
:10A9D0002046FFF7F9FE064325F0005545F0A04557
:10A9E000E4E700BF0000115038B50446857E2DB164
:10A9F000FFF780FFA38A2BB9284638BD8178084825
:10AA000000F03AFB2046FFF723FF054618B101236B
:10AA100023770025F0E72046FFF7AEFFECE700BF05
:10AA2000C07D0010F0B585B005460F464378042B75
:10AA300046D009D9052B4ED0062B1AD1874A137858
:10AA40000133DBB2137014E0022B03D0032B10D1BF
:10AA5000002456E0824B1A7822F001021A701A780C
:10AA600022F002021A7000225A701A7822F00402B0
:10AA70001A707C4B1C686369EFF3108272B6D3E8DE
:10AA8000CF0F01210028FAD1C3E8401F0028F6D1DA
:10AA9000BFF35F8FA2612946204600F0E1FA6169A9
:10AAA000A3690022C1E88F2F83F31088002800F0EB
:10AAB000C4803A466978287800F0CEFA05B0F0BD37
:10AAC000674B1B7813F0010FF8D0654A137843F0F9
:10AAD00004031370CDE7624B1B7813F0010FEDD028
:10AAE0005F4A137823F004031370C2E7D21A5E4B57
:10AAF00003EB4213DB6913B1696828789847013486
:10AB0000E4B25A4B1B782246591CA14207DBA342F0
:10AB1000ECD9574B1B6813EB4413EBD1EFE7504BC9
:10AB20001B7813F0040F33D14D4BDB7813F0010F7A
:10AB3000C4D02B788DF8043003238DF805306B6872
:10AB40000293484B1C686369EFF3108272B6D3E836
:10AB5000CF0F01210028FAD1C3E8401F0028F6D109
:10AB6000BFF35F8FA26101A9204600F079FA616905
:10AB7000A3690022C1E88F2F83F3108800284CD0EE
:10AB80003A469DF805109DF8040000F065FA95E737
:10AB9000334A137823F00403137001A900260196A9
:10ABA0004E608E602B788DF8043005238DF80530CB
:10ABB0002C4B1C686369EFF3108272B6D3E8CFCFD9
:10ABC0000120BCF1000FF9D1C3E84C0FBCF1000F1C
:10ABD000F4D1BFF35F8FA261204600F041FA6269B1
:10ABE000A369C2E88F6F83F3108838B13A469DF8A5
:10ABF00005109DF8040000F02FFA95E740F2651269
:10AC00001C491D4800F03CFA4FF0E023D3F8F03D1A
:10AC100013F0010F88D000BE86E740F26512154997
:10AC2000154800F02DFA4FF0E023D3F8F03D13F073
:10AC3000010F3FF443AF00BE40E740F265120D49FB
:10AC40000D4800F01DFA4FF0E023D3F8F03D13F06B
:10AC5000010F3FF433AF00BE30E700BFDF1E00201E
:10AC6000141400206C140020A0820010DD1E0020AF
:10AC7000441200201C820010207E001000B5844683
:10AC800010464FF0000E0AE0DCF80C3013F0020F13
:10AC9000FAD011F80E30CCF808300EF1010E8645CE
:10ACA000F2D301E0DCF80830DCF80C3013F0040FCC
:10ACB000F8D1DCF80C3013F0100FFAD101E0DCF819
:10ACC0000830DCF80C3013F0040FF8D10123CCF875
:10ACD000203000BD53B94AB9002908BF00281CBF65
:10ACE0004FF0FF314FF0FF3000F0ACB9ADF1080C80
:10ACF0006DE904CE00F006F8DDF804E0DDE902239A
:10AD000004B070472DE9F047064682B01746084662
:10AD10000A9AB4460D46002B4DD18F42BE4665D9E6
:10AD2000B7FA87F149B1C1F120038D4007FA01FE5E
:10AD300006FA01FC26FA03F31D434FEA1E461FFAEA
:10AD40008EF04FEA1C43B5FBF6F406FB145543EABC
:10AD5000054304FB00F59D4206D91EEB030302D216
:10AD60009D4200F24C81013C5B1B1FFA8CFCB3FB43
:10AD7000F6F506FB153305FB00F04CEA034C604585
:10AD80000AD91EEB0C0C2CBF01230023604502D90D
:10AD9000002B00F03781013DACEB000C45EA04408C
:10ADA000002422B12CFA01F30021C2E9003121462E
:10ADB00002B0BDE8F0878B4208D90AB1C2E9006150
:10ADC00000242046214602B0BDE8F087B3FA83F4A0
:10ADD000002C4DD18B42C0F00581B74240F2028178
:10ADE0002046002AE3D0C2E900C5E0E7002F00F0CA
:10ADF000A2801946B7FA87F3002B40F0B480C31B3A
:10AE00001FFA8EF83F0C01244FEA1C40B3FBF7F504
:10AE100007FB153340EA034308FB05F098420AD9C3
:10AE20001EEB03032CBF01260026984202D9002EF8
:10AE300000F0E280013D1B1A1FFA8CFCB3FBF7F017
:10AE400007FB10334CEA034C08FB00F363450AD9B7
:10AE50001EEB0C0C2CBF01260026634502D9002EE8
:10AE600000F0C7800138ACEB030C40EA054098E7DE
:10AE7000C4F12008A34006FA04FAA14027FA08FC0E
:10AE800020FA08F007FA04F94CEA030C26FA08F352
:10AE90004FEA1C460B431FFA8CFE190CB0FBF6F769
:10AEA00006FB170041EA004107FB0EF088420AD971
:10AEB0001CEB01012CBF01250025884202D9002D81
:10AEC00000F0B280013F091A9BB2B1FBF6F006FB1D
:10AED000101100FB0EFE43EA01439E450AD91CEB0C
:10AEE00003032CBF012100219E4502D9002900F057
:10AEF0009E80013840EA0740A3EB0E03A0FB09E166
:10AF00008B4276460F4602D307D1F24505D2BEEBFF
:10AF1000090661EB0C0101380F4652B1BAEB06018C
:10AF200063EB070303FA08F5E140E3400D43C2E990
:10AF3000005300243BE77308B8464908019743EAE9
:10AF4000C0734FEAC67C1C0C9BB244EA014443EA3E
:10AF50000443B4FBF7F4B1FBF7F51F21019844EA71
:10AF600005441B1A50E7194607FA03FEC3F12003F4
:10AF700000FA01F44FEA1E47D84026FA03F31FFAFD
:10AF80008EF806FA01FC2343B0FBF7F51C0C07FB17
:10AF9000150044EA004005FB08F484424AD91EEB40
:10AFA00000002CBF01260026844200D98EB3001B6E
:10AFB000013DB0FBF7F404FB08F6A146019607FB40
:10AFC00019009BB2019E43EA0043B342C6D21EEB76
:10AFD00003032CBF01200020B34200D2A8B109F125
:10AFE000FF34BBE7B6EB070C60EB030301201D4603
:10AFF000F7E6F444023836E7023D73441BE7023CAF
:10B000007344B1E6F444023DC6E6A9F10204734478
:10B01000A4E7AEEB0404023D2044B0FBF7F404FBCC
:10B0200008F6A1460196CAE7023F61444BE70238A1
:10B0300063445FE7001BB0FBF7F404FB08F6A1468E
:10B040000196BCE7704700BF5FF800F03D7100104B
:10B050005FF800F0ED1200105FF800F0953E001070
:10B060005FF800F0936000105FF800F0653B00109F
:10B070005FF800F0791400105FF800F0D5040010BC
:10B080005FF800F08D3100105FF800F0CD2E001059
:10B09000100000000000000000000100000000009F
:10B0A000000000000000020000000000000000009E
:10B0B0000000030000000000000000000000FF008E
:10B0C0000000000001B5486801318E460047704617
:10B0D00009380149884701BD110A0010000000002D
:10B0E0000000000000000000000000000000000060
:10B0F000080F002011360010B5320010793500100D
:10B10000A1320010000000000001000070140020B7
:10B1100010000C0000000000000000000000000013
:10B120000000000000000000FF00000040120020AE
:08B13000000000000000000017
:10B13800D3DEFFFFFE010000FF0100000050FFFF0B
:04B14800793512AB98
:040000051000014D99
:00000001FF
